:020000040000FA
:04000000A2EF03F078
:0400080005EF19F0F7
:080018008AEF19F00F0B6D6F68
:10002000000EF76E360EF66E6D51F626D8B0F72A32
:100030000800F55012003031323334353637383954
:100040004142434445468A86FA0E306E09841200C6
:100050008A96306A09941200000EF86E340EF76E1C
:100060002A0EF66EE4EC13F075EC1CF0B5EC00F023
:1000700003E3446A456A04D077C044F078C045F091
:10008000F8EC1EF06FEC20F057EC23F0EFEC26F0CC
:10009000030E636F010E646F91EC26F0E2EC25F025
:1000A000000EF86E380EF76EE20EF66EE8EC13F006
:1000B000000EF86E340EF76E240EF66EE4EC13F0BC
:1000C00075EC1CF0B5EC00F003E3446A456A04D01B
:1000D00079C044F07AC045F0F8EC1EF06FEC20F0E7
:1000E00057EC23F0EFEC26F0040E636F020E646F02
:1000F00091EC26F0E2EF25F0000EF86E340EF76E6C
:100100001C0EF66EE4EC13F075C044F076C045F0BA
:10011000CAEC1EF06FEC20F057EC23F059C0AAF1A6
:100120005AC0ABF15BC0ACF15CC0ADF15DC0AEF1EB
:1001300049EC28F0BEEC28F0B5EC00F013E3446A7B
:10014000456A466A476A486A44C0AFF145C0B0F1A3
:1001500046C0B1F147C0B2F148C0B3F1030E446EDE
:1001600044C0B9F18EEC2AF01200766703D07567AF
:1001700001D002D0D89076BFD8801200906703D00B
:100180008F6701D002D0D89090BFD8801200BFEC0A
:1001900001F028EC03F0E6EC02F058EC00F02CEC57
:1001A00000F07CEC00F07C6703D0ADEC02F0DDD019
:1001B000010E7C6309D0000EF86E360EF76ECC0E81
:1001C000F66EE4EC13F0CFD0020E7C6309D0000E83
:1001D000F86E360EF76EE20EF66EE4EC13F0C1D058
:1001E000030E7C6309D0000EF86E360EF76EF80E23
:1001F000F66EE4EC13F0B5D0040E7C630BD028EC63
:1002000000F0000EF86E370EF76E0E0EF66EE4EC90
:1002100013F0A7D0050E7C6309D0000EF86E370EE0
:10022000F76E240EF66EE4EC13F09BD0060E7C63A2
:1002300009D0000EF86E370EF76E3A0EF66EE4EC4B
:1002400013F08FD0070E7C630BD023EC00F0000E70
:10025000F86E370EF76E500EF66EE4EC13F081D0A8
:10026000080E7C6309D0000EF86E370EF76E660E2E
:10027000F66EE4EC13F075D0090E7C630BD023EC22
:1002800000F0000EF86E370EF76E7C0EF66EE4ECA2
:1002900013F069D00A0E7C6325D023EC00F0000E29
:1002A000F86E370EF76E920EF66EE4EC13F083ECF8
:1002B0001CF093C044F0D7EC26F0020E636FB6EC4E
:1002C00025F02D0E43EC13F083EC1CF094C044F0A9
:1002D000D7EC26F0020E636FB6EC25F02D0E43EC42
:1002E00013F041D00B0E7C630BD028EC00F0000E15
:1002F000F86E370EF76EA00EF66EE4EC13F031D008
:100300000C0E7C630BD028EC00F0000EF86E370E5C
:10031000F76EB60EF66EE4EC13F023D0140E7C6389
:100320001ED0000EF86E370EF76ECC0EF66EE4ECB3
:1003300013F075EC1CF083C044F0D7EC26F0030EEC
:10034000636F646BB6EC25F0000EF86E370EF76E37
:10035000DE0EF66EE8EC13F0D2EC13F004D0D8EC1D
:1003600011F0D8EC11F0030E2A6E08B848EC07F033
:1003700008BA3BEC07F008BC2EEC07F01200000EA8
:10038000F86E330EF76EFA0EF66EE4EC13F075ECC1
:100390001CF089C044F08AC045F0D7EC26F0030E6B
:1003A000636FE2EC25F0000EF86E330EF76EFE0E72
:1003B000F66EE4EC13F075EC1CF088C044F0D7EC5A
:1003C00026F0030E636FE2EC25F0876710D0000E75
:1003D000F86E340EF76E300EF66EE4EC13F0000E8D
:1003E000F86E340EF76E360EF66EE4EC13F0010E76
:1003F000876310D0000EF86E340EF76E3C0EF66E6A
:10040000E4EC13F0000EF86E340EF76E420EF66E4A
:10041000E4EC13F0020E876310D0000EF86E340E79
:10042000F76E480EF66EE4EC13F0000EF86E340E24
:10043000F76E4E0EF66EE4EC13F0030E876310D0E9
:10044000000EF86E340EF76E540EF66EE4EC13F0F8
:10045000000EF86E340EF76E5A0EF66EE4EC13F0E2
:10046000040E876310D0000EF86E340EF76E600E27
:10047000F66EE4EC13F0000EF86E340EF76E660EB6
:10048000F66EE4EC13F0050E876310D0000EF86EE4
:10049000340EF76E6C0EF66EE4EC13F0000EF86E90
:1004A000340EF76E720EF66EE4EC13F01200000ECE
:1004B000F86E340EF76E0A0EF66EE4EC13F0A5C17A
:1004C00059F0A6C15AF0A7C15BF0A8C15CF0A9C160
:1004D0005DF0EFEC26F0050E636F010E646F91EC9A
:1004E00026F0E2EC25F0040E43EC13F0000EF86E5B
:1004F000340EF76E160EF66EE4EC13F09BC159F055
:100500009CC15AF09DC15BF09EC15CF09FC15DF043
:10051000EFEC26F0050E636F010E646F91EC26F090
:10052000E2EC25F0D2EC13F0A0C159F0A1C15AF0D1
:10053000A2C15BF0A3C15CF0A4C15DF0EFEC26F0BA
:10054000050E636F010E646F668591EC26F0E2EC98
:1005500025F06A0E43EC13F01200540ED0EC13F0A9
:10056000460E43EC13F009B603D09651300901D082
:10057000700E43EC13F03A0E43EC13F075EC1CF0E4
:100580008BC044F08CC045F00A0E496E77EC24F025
:10059000D7EC26F0050E636F030E646FB6EC25F002
:1005A00009A602D009B809D0000EF86E340EF76E15
:1005B000780EF66EE8EC13F008D0000EF86E340EEC
:1005C000F76E7C0EF66EE8EC13F01200336608D07E
:1005D000000EF86E330EF76ECA0EF66EE4EC13F0F2
:1005E000010E336208D0000EF86E330EF76ED20E95
:1005F000F66EE4EC13F0030E336208D0000EF86ED2
:10060000330EF76EDA0EF66EE4EC13F0040E33627E
:1006100008D0000EF86E330EF76EE20EF66EE4ECC4
:1006200013F0020E336208D0000EF86E330EF76E30
:10063000EA0EF66EE4EC13F0050E336208D0000EFD
:10064000F86E330EF76EF20EF66EE4EC13F0120055
:10065000000EF86E340EF76E200EF66EE4EC13F01A
:1006600075EC1CF086C044F0D7EC26F0010E636FE9
:10067000E2EF25F0696F670ED0EC13F0695143EF9C
:1006800013F07C512FE1600ED0EC13F0D2EC13F09C
:100690005B0E43EC13F010EE11F0050E696FE6CF20
:1006A00044F00A0E446203D02A0E446E13D00B0E9F
:1006B000446203D0300E446E0DD00C0E446203D061
:1006C000230E446E07D0446603D02E0E446E02D033
:1006D000300E4412445043EC13F0692FE0D75D0E06
:1006E00043EC13F01200116A126A136A146A156A55
:1006F000166A10EE11F0E1CF0FF0E2CF10F01B6A96
:10070000120079EC03F00788190E1E6E078A088024
:100710000A0E276E1200806B816B21EEC7F0D9CFD5
:100720007EF0DACF7FF012000FC0E1FF10C0E2FFD1
:100730000DC0E6FFE1CF0FF0E2CF10F01B2A41EC35
:1007400003F01200F4EC11F0FAEC14F0EBEC14F0FE
:10075000BFEC12F056EC12F06EEC12F0C7EC00F0A9
:1007600073EC03F041EC03F07E0E4AEC12F0270E1E
:100770004AEC12F0080E4AEC12F048EC07F00A0EB0
:100780002D6E0888FA0E296E318CEFEC13F0D8A08C
:100790006DD1FA0E296E02EC14F00F0E0D64C0D06C
:1007A000C8EC13F0190E0D6221D0000EF86E340E55
:1007B000F76E920EF66EE4EC13F0000EF86E340E47
:1007C000F76EA20EF66EE4EC13F0000EF86E340E27
:1007D000F76EB80EF66EE4EC13F0000EF86E340E01
:1007E000F76ECE0EF66EE4EC13F07ED0180E0D62AE
:1007F00021D0000EF86E340EF76EE40EF66EE4ECC7
:1008000013F0000EF86E340EF76EF60EF66EE4EC92
:1008100013F0000EF86E350EF76E0C0EF66EE4EC6B
:1008200013F0000EF86E350EF76E220EF66EE4EC45
:1008300013F05AD0170E0D6219D0000EF86E350E57
:10084000F76E380EF66EE4EC13F0000EF86E350E0F
:10085000F76E4C0EF66EE4EC13F0000EF86E350EEB
:10086000F76E620EF66EE4EC13F03ED0160E0D62DB
:100870002DD0000EF86E350EF76E780EF66EE4ECA5
:1008800013F0AE51300943EC13F0000EF86E350E44
:10089000F76EC80EF66EE8EC13F0000EF86E350E2B
:1008A000F76E860EF66EE4EC13F0000EF86E350E61
:1008B000F76E9C0EF66EE4EC13F0000EF86E350E3B
:1008C000F76EB20EF66EE4EC13F00ED0000EF86E7A
:1008D000340EF76E880EF66EE4EC13F00DC0E8FFF0
:1008E0000F0B300943EC13F00DC00EF066EC14F062
:1008F000D8EC11F061EC14F002EC14F00DC0E8FF3C
:100900000F0B300943EC13F00E38F00B0E6E0D5048
:100910000F0B0E1207EC15F0C8EC13F00D6AA6D001
:100920000C0E0D6206D094EC03F0010E1B6216D083
:100930001ED094EC03F0010E1B6201D018D00A0EF9
:100940000D6205D07C6BC8EC13F007820BD0050E4E
:100950001B620CD00C0E0D6E94EC03F041EC03F016
:10096000ABEC07F073EC03F041EC03F07FD0070E23
:10097000116205D073EC03F08867880736D00A0E41
:10098000116206D073EC03F0882B01E188692DD049
:10099000080E116208D073EC03F0872B060E875DFA
:1009A00001E1876B22D0060E11620ED073EC03F0CA
:1009B000896703D08A6701D006D089078929D8B40E
:1009C0008A07D8B4895311D0090E116236D0830E2C
:1009D000446E030E456E8A51455C02E18951445CC8
:1009E000D8B403D0892BD8B48A2BBFEC01F07E0E8B
:1009F0004AEC12F0260E4AEC12F087C0E8FF4AECEF
:100A000012F048EC07F00A0E2D6E08887E0E4AECB4
:100A100012F0250E4AEC12F088C0E8FF4AEC12F002
:100A200048EC07F00A0E2D6E0888DBEC06F073EC3C
:100A300003F08A80320E2C6E19D00C0E116216D083
:100A4000FAEC06F07E0E4AEC12F0270E4AEC12F099
:100A5000080E4AEC12F048EC07F00A0E2D6E0888DA
:100A600073EC03F08A80320E2C6E00D007BE06D0E5
:100A7000A8EC12F0D8A002D0B4EC0FF091EC12F078
:100A800032E3806706D0AA0EA16303D08BEC03F09B
:100A90002AD0806702D0A1C082F08251805DD8B098
:100AA00003D0A1C0E8FF811B7EC0D9FF7FC0DAFF61
:100AB000A1C0DEFFD9CF7EF0DACF7FF0802B80514E
:100AC000825DD8B00FD0A151815DD8A409D008862D
:100AD0008A80320E2C6E3BEC07F00A0E2E6E088ACE
:100AE0008BEC03F000D008A630D001EEC7F0EECFBB
:100AF00082F082078207EECF7CF0140E7C6115D065
:100B00000F0E826312D010EE86F0EECFE6FF822F3A
:100B1000FCD77C6709D093C095F094C096F0946799
:100B200002D0098601D0099608D0140E7C6305D046
:100B3000EECF83F0FA0E296E00D00896078221EEE0
:100B4000C7F0D9CF7EF0DACF7FF0314E318C010E75
:100B5000316207D007A205D0C7EC00F041EC03F0EA
:100B60000792020E31621AD007AE18D05BEC10F07B
:100B70002EEC07F00A0E2F6E088C0988079EA36BD7
:100B8000010E33620BD0600ED0EC13F02A0E07A6D4
:100B9000200E43EC13F00776C80E226E030E31626E
:100BA00012D0030E336206D0266604D02668C8EC45
:100BB00014F009D0050E336206D0266604D0320E3A
:100BC000266EB1EC14F0040E316207D008A005D0F7
:100BD000276603D008907BEC0EF0050E316207D03B
:100BE00008A805D02D6603D0089844EC07F0060E3F
:100BF000316207D008AA05D02E6603D0089A37ECD8
:100C000007F0070E316203D0226601D00894080E67
:100C100031620BD0010E336208D0236606D008A4DF
:100C200004D0D5EC14F0640E236E090E316211D09D
:100C3000010E33620ED023660CD008B40AD0E0EC6B
:100C400014F0E0EC11F0D5EC14F0640E236EC80E35
:100C5000226E0A0E31620ED021660CD007A00AD097
:100C6000C5C184F0C6C185F04EEC07F0079008803E
:100C70000A0E276E0B0E31622ED009B602D096A155
:100C80002AD007B028D08BC044F08CC045F0C5C135
:100C900049F0C6C14AF0B80E4B6E0B0E4C6E4A506E
:100CA0004C5C02E149504B5CD8A015D0AA0E4B6EAB
:100CB000000E4C6E4A504C5C02E149504B5CD8B07F
:100CC0000AD04A50455C02E14950445CD8B403D094
:100CD000320E216E07800C0E316207D008AC05D0B1
:100CE0002F6603D0089C2AEC07F00D0E316217D056
:100CF000296615D02A662A062A520FE17C6B7E0EE1
:100D00004AEC12F0270E4AEC12F0080E4AEC12F0F0
:100D100048EC07F00A0E2D6E0888FA0E296E0E0EAA
:100D2000316213D01E6611D007A805D073EC03F012
:100D300041EC03F0079807AA08D0079A14EC07F0D3
:100D400008A203D0B2EC0DF008920F0E316213D05E
:100D5000BEEC00F010E27C6707D09051765D02E1B6
:100D60008F51755DD8B007D052D8EE0E1F6E020EAF
:100D7000206E098000E3100E316211D009A00FD05F
:100D800020660DD01F660BD0756B766B8DC079F029
:100D90008EC07AF091C077F092C078F00990110E71
:100DA000316207D009A405D0306603D028EC00F0EA
:100DB0008A96C5EF03F07E0E4AEC12F0240E4AEC40
:100DC00012F089C0E8FF4AEC12F048EC07F00A0E76
:100DD0002D6E08887E0E4AEC12F0230E4AEC12F0BB
:100DE0008AC0E8FF4AEC12F048EC07F00A0E2D6EBC
:100DF00008881200756B766B776B786B796B7A6B02
:100E00008F6B906B916B926B8D6B8E6B12008FC0A2
:100E100075F090C076F08DC079F08EC07AF091C0F8
:100E200077F092C078F012002A6A7C6B7E0E4AEC52
:100E300012F0270E4AEC12F0080E4AEC12F048ECC1
:100E400007F00A0E2D6E0888FA0E296E12000A0E9F
:100E5000D0EF13F0FCDF200E43EF13F0F8DF2A0E83
:100E600008AE43EC13F012001E0ED0EF13F0FCDFBF
:100E7000200E43EF13F0F8DF2A0E08AE43EC13F018
:100E800012004A0ED0EF13F0FCDF200E43EF13F0F8
:100E9000F8DF2A0E08AE43EC13F0120075EC1CF0DC
:100EA00084C044F085C045F0E80E496E030E4A6EDA
:100EB00077EC24F0D7EC26F009B63D8E7E0E4AEC96
:100EC00012F0790E4AEC12F03D504AEC12F048EC68
:100ED00007F00A0E2D6E08887E0E4AEC12F07A0E8C
:100EE0004AEC12F03C504AEC12F048EC07F00A0EC3
:100EF0002D6E08887E0E4AEC12F07B0E4AEC12F042
:100F00003B504AEC12F048EC07F00A0E2D6E0888B0
:100F10007E0E4AEC12F07C0E4AEC12F03A504AEC8B
:100F200012F048EC07F00A0E2D6E08881200030E2E
:100F3000696F00EE13F004D0060E696F00EE11F039
:100F4000EFCF44F00B0E446201D0446A44C0EEFF80
:100F5000692FF6D71200088EFAEC06F00B0E11621C
:100F600001D003D0040E116033D0E6DF75EC1CF025
:100F700015C03AF014C03BF013C03CF012C03DF075
:100F800011C03EF0A4EC27F0D5EC1FF03AC044F0BD
:100F90003BC045F03CC046F03DC047F03EC048F085
:100FA0008AEC1CF00A0E496EEBEC24F044C0C5F14B
:100FB00045C0C6F144C084F045C085F04EEC07F052
:100FC00008800A0E276E73EC03F007824DEF0CF0D9
:100FD000113A12501112ABDF1B061B061B0675ECF3
:100FE0001CF0010E1B6203D013C03AF011D0020EA8
:100FF0001B6205D014C03AF013C03BF009D0030EB9
:101000001B6206D015C03AF014C03BF013C03CF090
:10101000A4EC27F0D5EC1FF03AC01CF03BC01DF04B
:10102000C8EC13F04B0E116224D009B622D01B6617
:1010300020D07E0E4AEC12F0270E4AEC12F01E0E63
:101040004AEC12F048EC07F00A0E2D6E0888000EEC
:10105000F86E180EF76EE60EF66EE4EC13F0000E66
:10106000F86E180EF76EFC0EF66EE4EC13F04CEF13
:101070000CF0410E116214D0010E1B6211D07E0ED5
:101080004AEC12F0260E4AEC12F01CC0E8FF4AECC3
:1010900012F048EC07F00A0E2D6E08884DEF0CF0A8
:1010A000420E116212D01B5210E07E0E4AEC12F07A
:1010B000250E4AEC12F01CC0E8FF4AEC12F048EC96
:1010C00007F00A0E2D6E0888E8D3430E116209D08E
:1010D0001B5207E01CC089F01DC08AF0DBEC06F053
:1010E000DCD3440E11621DD0010E1B621AD0600EBB
:1010F0001C267E0E4AEC12F0220E4AEC12F01CC0A6
:10110000E8FF4AEC12F048EC07F00A0E2D6E088852
:10111000000EF86E190EF76E120EF66EE4EC13F078
:10112000BBD309B6A0D0450E116263D01B6627D091
:101130007E0E4AEC12F0270E4AEC12F00A0E4AEC30
:1011400012F048EC07F00A0E2D6E0888000EF86EBB
:101150001A0EF76EE00EF66EE4EC13F0000EF86E69
:10116000190EF76E280EF66EE4EC13F0000EF86E12
:10117000190EF76E3E0EF66EE4EC13F08DD3010EF1
:101180001B6237D01C5235E00A0E1C6032D00A0EAA
:101190001C267E0E4AEC12F0270E4AEC12F01CC000
:1011A000E8FF4AEC12F048EC07F00A0E2D6E0888B2
:1011B000000EF86E1A0EF76EE00EF66EE4EC13F009
:1011C000000EF86E190EF76E280EF66EE4EC13F0B2
:1011D000000EF86E190EF76E3E0EF66EE4EC13F08C
:1011E000000EF86E190EF76E540EF66EE4EC13F066
:1011F00053D3020E1B6236D0133A14501312990EB9
:10120000136030D07E0E4AEC12F01F0E4AEC12F042
:1012100013C0E8FF4AEC12F048EC07F00A0E2D6EFE
:101220000888000EF86E1A0EF76EE00EF66EE4EC0B
:1012300013F0000EF86E190EF76E280EF66EE4EC41
:1012400013F0000EF86E190EF76E3E0EF66EE4EC1B
:1012500013F0000EF86E190EF76E6A0EF66EE4ECDF
:1012600013F01AD366D0450E116263D01B6627D0E7
:101270007E0E4AEC12F0270E4AEC12F00B0E4AECEE
:1012800012F048EC07F00A0E2D6E0888000EF86E7A
:101290001A0EF76EE00EF66EE4EC13F0000EF86E28
:1012A000190EF76E280EF66EE4EC13F0000EF86ED1
:1012B000190EF76E3E0EF66EE4EC13F0EDD2010E51
:1012C0001B6297D71C5235E00A0E1C6032D00B0E01
:1012D0001C267E0E4AEC12F0270E4AEC12F01CC0BF
:1012E000E8FF4AEC12F048EC07F00A0E2D6E088871
:1012F000000EF86E1A0EF76EE00EF66EE4EC13F0C8
:10130000000EF86E190EF76E280EF66EE4EC13F070
:10131000000EF86E190EF76E3E0EF66EE4EC13F04A
:10132000000EF86E190EF76E540EF66EE4EC13F024
:10133000B3D209B6C4D0460E116264D023EC00F0DB
:10134000000EF86E190EF76E800EF66EE4EC13F0D8
:10135000000EF86E190EF76E960EF66EE4EC13F0B2
:101360001B6617D07E0E4AEC12F0270E4AEC12F0E4
:10137000010E4AEC12F048EC07F00A0E2D6E0888B8
:10138000000EF86E190EF76EAC0EF66EE4EC13F06C
:1013900083D2010E1B6236D01C6617D07E0E4AEC3B
:1013A00012F0270E4AEC12F0020E4AEC12F048EC52
:1013B00007F00A0E2D6E0888000EF86E190EF76EF3
:1013C000C20EF66EE4EC13F067D2080E1C601AD061
:1013D000020E1C267E0E4AEC12F0270E4AEC12F08A
:1013E0001CC0E8FF4AEC12F048EC07F00A0E2D6E24
:1013F0000888000EF86E190EF76ED80EF66EE4EC43
:1014000013F04AD2470E11622BD023EC00F01B667A
:1014100027D07E0E4AEC12F0270E4AEC12F0000E96
:101420004AEC12F048EC07F00A0E2D6E0888000E08
:10143000F86E190EF76E800EF66EE4EC13F0000EE7
:10144000F86E190EF76EEE0EF66EE4EC13F0000E69
:10145000F86E1A0EF76E040EF66EE4EC13F01CD262
:10146000480E11622BD023EC00F01B6627D07E0EB5
:101470004AEC12F0270E4AEC12F0140E4AEC12F06D
:1014800048EC07F00A0E2D6E0888000EF86E190E53
:10149000F76E800EF66EE4EC13F0000EF86E190E87
:1014A000F76E960EF66EE4EC13F0000EF86E1A0E60
:1014B000F76E1A0EF66EE4EC13F0EED1C2D0460EC3
:1014C000116273D023EC00F0000EF86E190EF76E67
:1014D000800EF66EE4EC13F0000EF86E1A0EF76E46
:1014E000300EF66EE4EC13F01B660FD07E0E4AEC65
:1014F00012F0270E4AEC12F0020E4AEC12F048EC01
:1015000007F00A0E2D6E0888C7D1010E1B6219D094
:101510001C6617D07E0E4AEC12F0270E4AEC12F031
:10152000030E4AEC12F048EC07F00A0E2D6E088804
:10153000000EF86E1A0EF76E460EF66EE4EC13F01F
:10154000ABD1010E1C6217D07E0E4AEC12F0270EB2
:101550004AEC12F0040E4AEC12F048EC07F00A0EC6
:101560002D6E0888000EF86E1A0EF76E5C0EF66E81
:10157000E4EC13F091D1020E1C6217D07E0E4AECFF
:1015800012F0270E4AEC12F0050E4AEC12F048EC6D
:1015900007F00A0E2D6E0888000EF86E1A0EF76E10
:1015A000720EF66EE4EC13F077D1470E116223D081
:1015B00023EC00F01B661FD07E0E4AEC12F0270EC3
:1015C0004AEC12F0000E4AEC12F048EC07F00A0E5A
:1015D0002D6E0888000EF86E190EF76E800EF66EEE
:1015E000E4EC13F0000EF86E1A0EF76E880EF66E2D
:1015F000E4EC13F051D1480E116223D023EC00F03B
:101600001B661FD07E0E4AEC12F0270E4AEC12F039
:10161000010E4AEC12F048EC07F00A0E2D6E088815
:10162000000EF86E190EF76E800EF66EE4EC13F0F5
:10163000000EF86E1A0EF76E9E0EF66EE4EC13F0C6
:101640002BD1490E116229D01B6627D07E0E4AECA1
:1016500012F0270E4AEC12F0090E4AEC12F048EC98
:1016600007F00A0E2D6E0888000EF86E1A0EF76E3F
:10167000E00EF66EE4EC13F0000EF86E1A0EF76E44
:10168000B40EF66EE4EC13F0000EF86E1A0EF76E60
:10169000CA0EF66EE4EC13F0FFD0510E116228D0A2
:1016A000010E1B6225D01C5223E0060E1C6020D0C8
:1016B0007E0E4AEC12F0220E4AEC12F01CC0E8FF3B
:1016C0004AEC12F048EC07F00A0E2D6E0888000E66
:1016D000F86E1A0EF76EE00EF66EE4EC13F0000EE4
:1016E000F86E1A0EF76EF60EF66EE4EC13F0D4D028
:1016F000520E11622CD0020E1B6229D0133A1450E4
:101700001312110E136423D0550E136020D07E0ED9
:101710004AEC12F0220E4AEC12F013C0E8FF4AEC39
:1017200012F048EC07F00A0E2D6E0888000EF86ED5
:101730001A0EF76EE00EF66EE4EC13F0000EF86E83
:101740001B0EF76E0C0EF66EE4EC13F0A5D009B686
:101750001FD0530E11621CD0010E1B6219D01C66E3
:1017600002D0010E1C6E030E1C6402D0010E1C6E12
:101770007E0E4AEC12F0210E4AEC12F01CC0E8FF7B
:101780004AEC12F048EC07F00A0E2D6E088885D05E
:10179000540E116253D0010E1B6250D0090E1C6210
:1017A00021D009B61FD07E0E4AEC12F0270E4AEC6B
:1017B00012F01F0E4AEC12F048EC07F00A0E2D6EE4
:1017C0000888000EF86E1A0EF76EE00EF66EE4EC66
:1017D00013F0000EF86E1B0EF76E220EF66EE4ECA0
:1017E00013F05AD0070E1C6224D009B622D083EC25
:1017F0000FF01EE27E0E4AEC12F0270E4AEC12F0B9
:10180000200E4AEC12F048EC07F00A0E2D6E088804
:10181000000EF86E1A0EF76EE00EF66EE4EC13F0A2
:10182000000EF86E1B0EF76E380EF66EE4EC13F039
:1018300033D01C6603D0DAEC0EF02FD0550E1162B7
:1018400003D01CEC0FF029D0560E116225D009B63A
:1018500023D0000EF86E190EF76E800EF66EE4ECD3
:1018600013F0000EF86E1B0EF76E4E0EF66EE4ECE3
:1018700013F0020E1B6210D07E0E4AEC12F0200E06
:101880004AEC12F01CC0E8FF4AEC12F048EC07F0FA
:101890000A0E2D6E088801D007D881EC03F0C8EC41
:1018A00013F00782089E1200AE531CE0040EAE63D4
:1018B00005D0D7EC11F0D7EC11F014D0030EAE63C5
:1018C00005D0D8EC11F0D7EC11F00CD0020EAE63BD
:1018D00003D0D7EC11F006D0010EAE6303D0D8ECE4
:1018E00011F000D01200003D3D3D3D3D20466972A3
:1018F0006D77617265203D3D3D3D3D004052657311
:1019000065742C2073746172746574206E65752122
:101910002000003D20416E74656E6E652077616524
:10192000686C656E203D3D00402D204C2F43207596
:101930002E204C432D56617220696D202000142DFD
:101940002031306B487A205365676D656E74207363
:10195000617665005420202B2F2D20232078203104
:10196000306B487A202020202000545B343561629F
:101970005D20612D20622B287831306B487A290058
:10198000003D3D3D3D3D3D3D204D61746368203D42
:101990003D3D3D3D3D004020206E616368737469AC
:1019A0006D6D656E206175662020200040202061ED
:1019B0007566206B6C65696E73746573205357523E
:1019C0002000142020466C616563686520387838F3
:1019D000204C784320202000142020535752206BA5
:1019E0006C65696E657220312C78202020004020C3
:1019F000206E65752061627374696D6D656E20205F
:101A000020202000142020766F6C6C20696D20430C
:101A10002D5365676D656E7420001420206D696E0E
:101A20002E53575220696D20432D5365672E200099
:101A3000402D2052654D61746368202D2D2D2D2D74
:101A40002D2D2D2D2D00402D2052654D6174636884
:101A50002064656570202D2D2D2D2D00402D2052E8
:101A6000654D6174636820347834202D2D2D2D2D23
:101A70002D00402D2052654D617463682038783800
:101A8000202D2D2D2D2D2D00402D204D61746368AE
:101A9000202D2D2D2D2D2D2D2D2D2D2D2D00402D9D
:101AA000204D617463682064656570202D2D2D2D97
:101AB0002D2D2D004045696E7374656C6C756E67D5
:101AC000207370656963682E200014667565722046
:101AD0006461732067616E7A652042616E642000E4
:101AE000003D3D2045787465726E657220456570D5
:101AF000726F6D203D0040416E74656E6E652023EF
:101B0000206C6F65736368656E20200040416E74C1
:101B1000656E6E65206162206B6F70696572656EBF
:101B2000200040456570726F6D50494320736176A7
:101B3000652065787445700040456570726F6D5022
:101B4000494320726573746F726520202000404DF8
:101B50006178696D616C65722054756E652D506594
:101B600067656C0075EC1CF089C044F08AC045F0D4
:101B7000640E496EEBEC24F044C06CF075EC1CF084
:101B800089C044F08AC045F0696B6C6702D06983F4
:101B90004DD0010E6C6305D0640E496E6981698376
:101BA00043D0020E6C6305D0C80E496E698169830B
:101BB0003BD0030E6C6307D02C0E496E010E4A6EAB
:101BC0006981698331D0040E6C6307D0900E496E31
:101BD000010E4A6E6981698327D0050E6C6307D0B8
:101BE000F40E496E010E4A6E698169831DD0060E9E
:101BF0006C6307D0580E496E020E4A6E6981698384
:101C000013D0070E6C6307D0BC0E496E020E4A6EED
:101C10006981698309D0080E6C6306D0200E496E75
:101C2000030E4A6E698100D0F3EC1FF069A106D063
:101C30000A0E446003D026EC0EF007D069A305D04D
:101C40005A0E446402D047EC0EF01200C8EC13F0B8
:101C500068EC0EF0000EF86E360EF76E6C0EF66E37
:101C6000E4EC13F0000EF86E360EF76E8A0EF66E88
:101C7000E4EC13F0000EF86E360EF76EB60EF66E4C
:101C8000E4EC13F0D5EC11F0C8EC13F01200C8EC42
:101C900013F068EC0EF0000EF86E360EF76E6C0E58
:101CA000F66EE4EC13F0000EF86E360EF76EA00E32
:101CB000F66EE4EC13F0000EF86E360EF76EB60E0C
:101CC000F66EE4EC13F0D5EC11F0C8EC13F0120052
:101CD000000EF86E360EF76E820EF66EE4EC13F020
:101CE00083EC1CF089C044F08AC045F0D7EC26F0A4
:101CF000B6EC25F0120019D8A9C0A5F0790EA46F92
:101D0000ACEC0EF0A8C0A5F07A0EA46FACEC0EF00F
:101D1000A7C0A5F07B0EA46FACEC0EF0A6C0A5F09A
:101D20007C0EA46FACEC0EF0120075EC1CF084C0BD
:101D300044F085C045F0E80E496E030E4A6E77EC1C
:101D400024F0D7EC26F03AC0A6F03BC0A7F03CC088
:101D5000A8F03DC0A9F012007E0EB7EC0EF0A4C0B2
:101D6000E8FFB7EC0EF0A5C0E8FFB7EF0EF0CD909E
:101D7000446E8A940ED8080E696F4432D8A08A94B3
:101D8000D8B08A8406D8692FF8D78A8402D8CD8043
:101D900012009E0E0A6E0A2EFED71200D7EC26F015
:101DA0003B50300943EC13F02E0E43EC13F03A5045
:101DB000DAEF13F0000EF86E350EF76ECE0EF66EFB
:101DC000E4EC13F0000EF86E350EF76EFA0EF66EB8
:101DD000E4EC13F009B609D0000EF86E360EF76E7B
:101DE000100EF66EE4EC13F008D0000EF86E360E0E
:101DF000F76E200EF66EE4EC13F095C044F0CEECD6
:101E00000EF0000EF86E360EF76E300EF66EE4EC45
:101E100013F06C0E446ECEEC0EF0C80E246E000E65
:101E2000256E256603D0246601D005D0EFEC13F0B3
:101E3000F8E302EC14F01200BFEC01F01FEC18F014
:101E4000EAEC18F039EC0FF05EEC0FF00DEC16F048
:101E500057EC02F0EE0E246E020E256E256603D0BE
:101E6000246601D005D0EFEC13F0F8E302EC14F097
:101E70001200000EF86E340EF76E020EF66EE4ECF1
:101E800013F005C259F006C25AF007C25BF008C24F
:101E90005CF009C25DF0EFEC26F0050E636F010EF9
:101EA000646F91EC26F0E2EC25F0000EF86E340E33
:101EB000F76E840EF66EE8EC13F01200000EF86E6A
:101EC000340EF76E060EF66EE4EC13F000C259F015
:101ED00001C25AF002C25BF003C25CF004C25DF0C2
:101EE000EFEC26F0050E636F030E646F91EC26F0A5
:101EF000E2EC25F0000EF86E340EF76E800EF66EF2
:101F0000E8EC13F01200000EF86E350EF76ECE0EF0
:101F1000F66EE4EC13F0000EF86E350EF76EE40E7C
:101F2000F66EE4EC13F0000EF86E360EF76E400E0F
:101F3000F66EE4EC13F0000EF86E360EF76E560EE9
:101F4000F66EE4EC13F002EC14F0090E0D6202D010
:101F5000D89001D0D880120023EE00F0A3C0D9FFA2
:101F60009BC0DFFFA32B1200050E33620DD0ACEC3B
:101F70000FF03B0E9B6302D0078E04D0FA0EA365D0
:101F800001D0078E4AEF10F0040E33620DD0ACEC96
:101F90000FF03B0E9B6302D0078E04D0FA0EA365B0
:101FA00001D0078E4AEF10F0020E33620DD0ACEC78
:101FB0000FF0FD0E9B6302D0078E04D0FA0EA365CE
:101FC00001D0078E4AEF10F0030E33620DD0ACEC57
:101FD0000FF03B0E9B6302D0078E04D0FA0EA36570
:101FE00001D0078E4AEF10F0010E336224D0A367B0
:101FF00003D09BC000F318D0010EA36303D09BC095
:1020000001F312D0020EA36303D09BC002F30CD0E5
:10201000030EA36303D09BC003F306D0040EA36397
:1020200003D09BC004F300D0A32B050EA36302D002
:10203000078E08842FD0000E33622CD07E0E9B5D5D
:1020400002E1A36B27D0A36704D09BC09CF0A32B15
:1020500021D0790E9C5D05E11ED81CE29BC0AAF040
:1020600019D07A0E9C5D05E116D814E29BC0ABF046
:1020700011D07B0E9C5D05E10ED80CE29BC0ACF04C
:1020800009D07C0E9C5D06E106D804E29BC0ADF051
:10209000078E00D012009B510F0B446E0A0E445C59
:1020A00008E29B51F00B446EA00E445C02E2D89013
:1020B0001200D8801200000E33621FD0AA53D8A499
:1020C00066EF10F0AB53D8B4AAEF11F083EC1CF01C
:1020D000ACC044F0ABC045F0AAC046F0D5EC1FF050
:1020E0007DEC1DF08AEC1CF00A0E496EEBEC24F03E
:1020F0003AC0C5F13BC0C6F12DD1010E336221D0EB
:1021000075EC1CF003C344F002C345F001C346F074
:1021100000C347F0D5EC1FF07DEC1DF08AEC1CF0FD
:102120000A0E496E77EC24F08AEC1CF0100E496E12
:10213000270E4A6EEBEC24F03AC0C5F13BC0C6F165
:1021400009D1030E336241D000C344F0460E44620D
:1021500001D101C344F0410E446201D003D0420ECC
:10216000446220D075EC1CF008C33AF007C33BF082
:1021700006C33CF005C33DF0A4EC27F0D5EC1FF0FE
:1021800001C344F0410E446205D03AC070F03BC038
:1021900071F019D0420E446205D03AC072F03BC0D3
:1021A00073F011D0540E44620ED002C374F0310E9D
:1021B000746305D072C0C5F173C0C6F104D070C09D
:1021C000C5F171C0C6F12668C5D0020E33623BD09E
:1021D00000C344F0FE0E4462BDD001C344F0FE0EC5
:1021E0004462B8D002C344F0000E4462B3D003C3CB
:1021F00044F0940E4462AED004C344F0000E446236
:10220000A9D00AC344F0FD0E4462A4D075EC1CF0C2
:1022100005C344F006C345F007C346F008C347F0C2
:1022200009C348F0D5EC1FF07DEC1DF08AEC1CF0E2
:10223000100E496E270E4A6EEBEC24F03AC0C5F141
:102240003BC0C6F187D0040E336262D000C344F0B5
:10225000460E44622ED001C344F0410E446201D0C8
:1022600003D0420E446251D00DC344F03B0E446291
:102270004CD075EC1CF008C33AF007C33BF006C322
:102280003CF005C33DF0A4EC27F0D5EC1FF001C3F2
:1022900044F0410E446205D03AC070F03BC071F08A
:1022A00021D0420E44627ED73AC072F03BC073F038
:1022B00019D05A0E446229D001C344F05A0E446228
:1022C00024D002C344F0530E44621FD003C344F031
:1022D000570E44621AD005C344F03B0E446215D039
:1022E00004C374F0746702D0300E746F310E7463DF
:1022F00005D072C0C5F173C0C6F107D0300E74634B
:1023000004D070C0C5F171C0C6F1A36BAAEF11F083
:10231000050E33621FD000C344F0460E446221D044
:1023200001C344F0410E44621CD075EC1CF006C39E
:102330003AF005C33BF004C33CF003C33DF0A4EC0A
:1023400027F0D5EC1FF03AC0C5F13BC0C6F1320E04
:10235000266E00D0C5C184F0C6C185F008800A0E83
:10236000276E1200140ED0EC13F083EC1CF070C03A
:1023700044F071C045F0D7EC26F0E2EC25F0540EA5
:10238000D0EC13F083EC1CF072C044F073C045F045
:10239000D7EC26F0E2EC25F0400ED0EC13F07451AF
:1023A00043EC13F0D8EC11F0120001D801D800D89A
:1023B00003D802D8DCEC11F0FA0E09D0C80E07D011
:1023C000640E05D0320E03D00A0E01D0010E0400B7
:1023D0000C6EFA0E0A6E060E0B6E0A2EFED70B2E30
:1023E000FCD70C2EF6D712000F01806A896A000E06
:1023F000386F1F0E926E816A8A6A000E396F000E66
:10240000936E826A8B6A800E946E000E3A6F836AB6
:102410008C6A800E956E000E3B6F846A8D6A000E8A
:102420003C6F070E966E000EC16EBE0EC06E000EA3
:10243000D06EC00EF26E400EF16E000EF06E010E08
:102440009D6E000EA06E220ED56E330ECD6E000E68
:10245000BA6E000EB16E0001000E816E800E826EAB
:10246000800E836E070E846E05D8D30ECF6E000EDD
:10247000CE6E1200696B00EE00F0EE6A692FFDD798
:10248000040E6A6F01EE00F0EE6A692FFDD76A2F25
:10249000FBD712000400A4A8FDD7736EE6EF11F07D
:1024A00004009EA8FDD7AD6EE6EF11F00400030E08
:1024B000336202D03B0E01D01D0EAF6E05EE00F070
:1024C000EACF98F0E9CF97F0EACF9AF0E9CF99F008
:1024D000AC94AC8AAB88AB8E9D8A1200040004EEEB
:1024E00000F0EACF9EF0E9CF9DF0EACFA0F0E9CF6F
:1024F0009FF01D0E756E7294728A7188718EA38A18
:10250000120004009EAA03D0AE50D8901200D880CA
:1025100012000400A4AA03D07450D8901200D880EE
:1025200012009FC0E1FFA0C0E2FF9D51E15C02E10B
:10253000D8901200E650A16FF10EE15C02E114EEBA
:1025400000F0E1CF9FF0E2CFA0F0A151D8801200BF
:1025500099C0E1FF9AC0E2FF9751E15C02E1D89097
:102560001200E6509B6FF10EE15C02E115EE00F007
:10257000E1CF99F0E2CF9AF09B51D880120080A66B
:102580001200809A83928390E2EC11F0200EA3EC6B
:1025900013F0800EA3EC13F0E4EC11F0200EA3EC8A
:1025A00013F0800EA3EC13F0E6EC11F0060E95ECA0
:1025B00013F00C0E95EC13F0140E95EC13F063EC85
:1025C00013F0E5EC12F0C8EF13F0C8EC13F0000EB6
:1025D000F86E370EF76EE00EF66EE4EC13F0000EB8
:1025E000F86E370EF76EF60EF66EE4EC13F0000E92
:1025F000F86E380EF76E0C0EF66EE4EC13F0000E6B
:10260000336208D0000EF86E380EF76E220EF66EAA
:10261000E4EC13F0010E336208D0000EF86E380EB1
:10262000F76E380EF66EE4EC13F0030E336208D04A
:10263000000EF86E380EF76E4E0EF66EE4EC13F0E8
:10264000040E336208D0000EF86E380EF76E640E7A
:10265000F66EE4EC13F0020E336208D0000EF86E52
:10266000380EF76E7A0EF66EE4EC13F0050E336258
:1026700008D0000EF86E380EF76E900EF66EE4EC91
:1026800013F0D7EF11F0346EB3EC13F034508382B3
:102690008390809AF00BA3EC13F03438F00B53D0F6
:1026A000346E344634463446B3EC13F034504009AB
:1026B00095EC13F0080E696F0900F55043EC13F028
:1026C000692FFAD7120080A61200000EF86E260EAF
:1026D000F76EEA0EF66E080E6A6F6B6B6B5150EC7C
:1026E00013F06B2B6A2FFAD7120000000E11110A9B
:1026F0001B0000001010100001150000141414003D
:10270000011500001515150001150E1111110A0A09
:102710001B0000000000000000000000000000009E
:102720000000000000000000000080A61200346ECF
:10273000B3EC13F03450F00B83928390809AA3ECA7
:1027400013F03438F00B80A61200E8380F0B82B873
:10275000100982BA200982BC400982BE8009826EBB
:10276000808A809A120080A61200828694868392C4
:1027700083806697808A000082A66687809A000020
:10278000808A0000809A66A7F4D7949683901200FE
:10279000010ECBD7020EC9D7800EC7D7C00EC5D742
:1027A0008009C3D7200E6FD7696FD2EC13F0692F61
:1027B000FCD71200356E35380EEC00F043EC13F008
:1027C00035500EEC00F05FD70900F550D0EC13F057
:1027D0000900F55003E043EC13F0FAD71200F8ECCF
:1027E00013F058EC14F002E0D88001D0D890120019
:1027F0008B808B828B848B8612008B908B928B9438
:102800008B961200EFEC13F0FDE30D6A34EC14F03C
:102810000D6E040E696FE4EC11F034EC14F00D62EF
:10282000F1D7692FF8D7000E0DB807D0030E0DBAF7
:1028300004D0060E0DBC01D0090E6A6F010E0DB456
:1028400004D0020E0DB201D0030E6A276AC00DF04B
:10285000500E696FEFEC13F006E3E4EC11F0692F12
:10286000F9D7100E0D261200FDEC13F08B8058ECFA
:1028700014F015E1FDEC13F08B8258EC14F00FE12D
:10288000FDEC13F08B8458EC14F009E1FDEC13F02F
:102890008B8658EC14F003E16A6BE86A12008250F0
:1028A000E838F00B6A6F58EC14F06A11FDEF13F082
:1028B0008450070BE8A002D0040E02D0E8B4010E49
:1028C00012000D6AEFEC13F0FCE31200EFEC13F0D2
:1028D000FDE212001D0E0DD0190E0BD0150E09D001
:1028E000110E07D00D0E05D0090E03D0050E01D034
:1028F000010EC26EC282C2B2FED7C4CF6FF0C3CF88
:102900006EF01200A6B2FED705C0A9FF06C0A8FF50
:10291000A69EA69CA684F29EF2BEFDD7550EA76E7B
:10292000AA0EA76EA68207A4F28EA6941200A6B2E3
:10293000FED705C0A9FFA69EA69CA680A8CF06F03C
:102940001200DECF06F082EC14F0052A692FF9D7C9
:10295000120097EC14F006C0DEFF052A692FF9D7A4
:102960001200460E50EC12F0410E50EC12F03B0EED
:1029700050EC12F01200410E50EC12F0490E50ECE7
:1029800012F0310E50EC12F03B0E50EC12F012002F
:10299000410E50EC12F0490E50EC12F0320E50EC99
:1029A00012F03B0E50EC12F01200010E336207D011
:1029B000A36B040E696F09D8030E50EF12F01200DA
:1029C000010E336207D0050E696FE86A50EC12F011
:1029D000692FFBD71200020E056E97EC14F006C0AB
:1029E000AEF01200AEC006F0020E056E82EC14F0DE
:1029F000E0EF11F0056A97EC14F006C033F0120016
:102A000033C006F0056A82EC14F0E0EF11F0910E8D
:102A10000E6203D0000E336E4CD0920E0E6203D0C5
:102A2000010E336E46D0930E0E6203D0020E336E4B
:102A300040D0940E0E6203D0030E336E3AD0950E42
:102A40000E6203D0040E336E34D0960E0E6203D0A5
:102A5000050E336E2ED08B0E0E6202D062EF15F093
:102A6000810E0E6202D0A2EF15F0710E0E6202D03E
:102A7000E2EF15F06B0E0E6202D0AE6B18D0610E55
:102A80000E6203D0010EAE6F12D0620E0E6203D042
:102A9000020EAE6F0CD0630E0E6203D0030EAE6F4B
:102AA00006D0640E0E6203D0040EAE6F00D09ADF23
:102AB00001D0A6DF07821200050E336202D0B1EC0E
:102AC00014F01200746BC8EC13F00D6A0E6AEFEC90
:102AD00013F00DE302EC14F00C0E0D6201D0FF00B8
:102AE0000B0E0D6204D0C8EC13F0E6DF746BA8EC9B
:102AF00012F0EBE3280E746301D0746B746705D099
:102B000095EC19F0000ED0EC13F00A0E746305D0AA
:102B10009EEC19F0400ED0EC13F0140E746305D047
:102B2000A7EC19F0140ED0EC13F01E0E746305D050
:102B3000B0EC19F0540ED0EC13F09B51DAEC13F01A
:102B4000742BC3D7746BC8EC13F00D6A0E6AEFECEC
:102B500013F00DE302EC14F00C0E0D6201D0FF0037
:102B60000B0E0D6204D0C8EC13F0A6DF746BA8EC5A
:102B700012F0EBE3500E746301D0746B746705D0F0
:102B800095EC19F0000ED0EC13F0140E746305D020
:102B90009EEC19F0400ED0EC13F0280E746305D0B3
:102BA000A7EC19F0140ED0EC13F03C0E746305D0B2
:102BB000B0EC19F0540ED0EC13F09B5143EC13F031
:102BC000742BC3D7746BC8EC13F0000EF86E350E7F
:102BD000F76E620EF66EE4EC13F00D6A0E6AEFEC1F
:102BE00013F01AE302EC14F01C0E0D6201D0FF008A
:102BF0000A0E0D6202D02A0E0DD00B0E0D6202D00D
:102C0000300E08D00C0E0D6202D0230E03D00DC082
:102C1000E8FF300943EC13F0E0D7EAEC18F01FECC2
:102C200018F075EC1CF08BC044F08CC045F0445299
:102C300004E1455202E11EEF18F0F8EC1EF06FECD3
:102C400020F0B7EC22F005EC21F0A8EC22F085ECA6
:102C500020F08AEC22F085EC20F059C02CF15AC00B
:102C60002DF15BC02EF15CC02FF15DC030F100C2D0
:102C700059F001C25AF002C25BF003C25CF004C218
:102C80005DF02CC15EF02DC15FF02EC160F02FC150
:102C900061F030C162F085EC20F059C091F15AC06A
:102CA00092F15BC093F15CC094F15DC095F105C2F7
:102CB00059F006C25AF007C25BF008C25CF009C2C4
:102CC0005DF02CC15EF02DC15FF02EC160F02FC110
:102CD00061F030C162F085EC20F059C022F15AC099
:102CE00023F15BC024F15CC025F15DC026F1D9EC75
:102CF00022F0ACEC1CF022C15EF023C15FF024C1D5
:102D000060F025C161F026C162F005EC21F05D8E16
:102D100059C096F15AC097F15BC098F15CC099F127
:102D20005DC09AF1010E876331D082EC22F05EC063
:102D30004BF15FC04CF160C04DF161C04EF162C01B
:102D40004FF191C150F192C151F193C152F194C12F
:102D500053F195C154F1596A5A6A5B6A5C6A5D6ABB
:102D600059C055F15AC056F15BC057F15CC058F1DB
:102D70005DC059F196C15AF197C15BF198C15CF100
:102D800099C15DF19AC15EF182EC2EF0020E87636B
:102D900044D0596A5A6A5B6A5C6A5D6A59C050F1EC
:102DA0005AC051F15BC052F15CC053F15DC054F1A7
:102DB00059C055F15AC056F15BC057F15CC058F18B
:102DC0005DC059F182EC22F05EC04BF15FC04CF166
:102DD00060C04DF161C04EF162C04FF196C15AF131
:102DE00097C15BF198C15CF199C15DF19AC15EF147
:102DF00082EC2EF00101556B566B576B586B596B7B
:102E0000000191C15AF192C15BF193C15CF194C18F
:102E10005DF195C15EF1ECEC2BF0030E876331D0D0
:102E200082EC22F05EC04BF15FC04CF160C04DF10E
:102E300061C04EF162C04FF196C150F197C151F19E
:102E400098C152F199C153F19AC154F1596A5A6A21
:102E50005B6A5C6A5D6A59C055F15AC056F15BC045
:102E600057F15CC058F15DC059F191C15AF192C15E
:102E70005BF193C15CF194C15DF195C15EF182ECAF
:102E80002EF0040E876344D0596A5A6A5B6A5C6A02
:102E90005D6A59C050F15AC051F15BC052F15CC03B
:102EA00053F15DC054F159C055F15AC056F15BC0A1
:102EB00057F15CC058F15DC059F182EC22F05EC060
:102EC0004BF15FC04CF160C04DF161C04EF162C08A
:102ED0004FF191C15AF192C15BF193C15CF194C180
:102EE0005DF195C15EF182EC2EF00101556B566BE0
:102EF000576B586B596B000196C15AF197C15BF142
:102F000098C15CF199C15DF19AC15EF1ECEC2BF0D6
:102F1000876716D082EC22F05EC04BF15FC04CF1A7
:102F200060C04DF161C04EF162C04FF191C150F1EE
:102F300092C151F193C152F194C153F195C154F131
:102F4000050E876316D082EC22F05EC04BF15FC0A5
:102F50004CF160C04DF161C04EF162C04FF196C1BD
:102F600050F197C151F198C152F199C153F19AC1F1
:102F700054F10101547F00014BC19BF14CC19CF104
:102F80004DC19DF14EC19EF14FC19FF150C1A0F1C5
:102F900051C1A1F152C1A2F153C1A3F154C1A4F195
:102FA0004BC159F04CC15AF04DC15BF04EC15CF0C1
:102FB0004FC15DF04BC15EF04CC15FF04DC160F0A0
:102FC0004EC161F04FC162F085EC20F059C00EF1A6
:102FD0005AC00FF15BC010F15CC011F15DC012F17D
:102FE00050C159F051C15AF052C15BF053C15CF06D
:102FF00054C15DF050C15EF051C15FF052C160F04C
:1030000053C161F054C162F085EC20F00EC15EF056
:103010000FC15FF010C160F011C161F012C162F028
:1030200048EC21F0B1EC21F059C0A5F15AC0A6F14D
:103030005BC0A7F15CC0A8F15DC0A9F1120075ECFE
:103040001CF089C044F08AC045F0F8EC1EF06FEC2B
:1030500020F0C2EC1CF089C044F08AC045F0640E38
:10306000496E000E4A6E4A50455C02E14950445C8C
:10307000D8B001D08DD0C80E496E000E4A6E4A50AD
:10308000455C02E14950445CD8B001D054D02C0ECC
:10309000496E010E4A6E4A50455C02E14950445C5B
:1030A000D8B001D048D0900E496E010E4A6E4A50F9
:1030B000455C02E14950445CD8B001D03CD0F40EEC
:1030C000496E010E4A6E4A50455C02E14950445C2B
:1030D000D8B001D030D0580E496E020E4A6E4A5018
:1030E000455C02E14950445CD8B001D024D0BC0E0C
:1030F000496E020E4A6E4A50455C02E14950445CFA
:10310000D8B001D018D0200E496E030E4A6E4A5036
:10311000455C02E14950445CD8B001D00CD0840E2B
:10312000496E030E4A6E4A50455C02E14950445CC8
:10313000D8B001D000D083EC1CF049C044F04AC0A4
:1031400045F0F8EC1EF06FEC20F0B7EC22F042EC0A
:1031500021F046EC1DF0B7EC22F042EC21F051ECEE
:103160001DF0A1EC1CF0D8EC1CF042EC21F03F0E5D
:10317000626FB30E616F330E606F330E5F6E330E8E
:103180005E6E85EC20F0EEEC1CF048EC21F00ED0E9
:10319000A1EC1CF03E0E626FBD0E616F700E606F91
:1031A000A30E5F6ED70E5E6E85EC20F0410E626F4F
:1031B000880E616F5E6A5F6A606B48EC21F059C0EF
:1031C00005F25AC006F25BC007F25CC008F25DC0AF
:1031D00009F2120075EC1CF088C044F0F8EC1EF007
:1031E0006FEC20F03E0E626F5E6A5F6A606B616B2F
:1031F00085EC20F059C000F25AC001F25BC002F227
:103200005CC003F25DC004F21200EACF04F0E9CF23
:1032100003F098C0EAFF97C0E9FF9EAA0ED0AE5017
:10322000ABA204D0AE50AB98AB88F7D7EE6EF10EE0
:10323000E95C02E105EE00F0F0D7EACF98F0E9CFC3
:1032400097F09EC0EAFF9DC0E9FFA4AA0ED074507B
:1032500071A204D0745071987188F7D7EE6EF10E98
:10326000E95C02E104EE00F0F0D7EACF9EF0E9CF8E
:103270009DF0F2A402D0F29448D0F2A202D0F292D1
:1032800044D09EA03AD09E902B662B062C662C062E
:103290002B668A922C668A901E661E06216621067F
:1032A0002266220623662306256602D0245206E003
:1032B00024062428D8B42506D8B42452206602D087
:1032C0001F5206E01F061F28D8B42006D8B41F528C
:1032D0002666260627662706286628062966290602
:1032E0002D662D062E662E062F662F0630663006BA
:1032F000D30ECF6E000ECE6E08D0A1A802D0A1983A
:1033000004D09EA202D09E9200D004C0EAFF03C067
:10331000E9FF1100006ED8CF01F0E0CF02F002C04B
:10332000E0FF005001C0D8FF1000000EF86E330E11
:10333000F76E720EF66EE4EC13F01200000EF86EEB
:10334000330EF76E880EF66EE4EC13F01200000EEA
:10335000F86E330EF76E9E0EF66EE4EC13F012006C
:10336000000EF86E330EF76EB40EF66EE4EC13F04A
:10337000120000202020202020202020202020209B
:10338000202020202020200040202020202020203D
:103390002020202020202020202020202000142059
:1033A000202020202020202020202020202020201D
:1033B00020202000542020202020202020202020F9
:1033C000202020202020202020000B5053746172E8
:1033D00000000B465438343700000B4B32202020BD
:1033E00000000B507753445200000A4943373330F2
:1033F00030000B4654445820000000433A00404C33
:103400003A000A433A004A4C3A0014496D70656428
:10341000616E7A3D2000545A3D20000014503A005D
:1034200011413A004B5357523A001F524C3A000098
:10343000062D4C2D0000462020200000062D4C2B90
:103440000000462020430000062B4C2D0000464380
:1034500020200000062D432B00004620204C0000B9
:10346000062B432D0000464C20200000062D432D46
:1034700000004620202000004D487A00636174005F
:1034800075480000704600000042656665686C3A49
:103490002000005452582052656D6F74653A2039EF
:1034A0000000405B315D505374617220205B345DDD
:1034B0004B32202020202000145B325D46543834EB
:1034C0003720205B355D5077534452202000545BF9
:1034D000335D494337333030205B365D46544458C2
:1034E00031303100005253323332204D6F6E6974E7
:1034F0006F723A203800405B305D20486578646523
:103500007A696D616C20202020202000145B315DE1
:103510002041736363692020202020202020202068
:103520002000545B235D2041626272756368202035
:103530002020202020202000005465737466756EC2
:103540006B74696F6E656E3A20370000405B315DC9
:103550002054617374656E66656C642020202020A1
:103560002000545B23206C616E675D2041626272B3
:10357000756368212120200000496E666F74696DB3
:1035800065723D200000405B305D20302053656B4C
:103590002E5B315D20312053656B2E00145B325D54
:1035A00020322053656B2E5B335D20332053656BD7
:1035B0002E00545B345D20342053656B2E5B235DFD
:1035C00020416262722E20002053656B2E00003D68
:1035D0003D3D3D3D2046756E6B74696F6E203D3DEF
:1035E0003D3D3D00402D206578746565202D2D3EC4
:1035F000205049436565202D2D00402D2D2D20465E
:10360000572056657273696F6E656E202D2D2D00E3
:103610001453796D54756E6572202020203A000095
:10362000145069634154553530302020203A000051
:103630005453796D54756E52656D6F74653A000020
:1036400014205B395D204F4B2057656974657220EB
:1036500020202020200054205B235D2041626272E4
:10366000756368202020202020202000004265660D
:103670002E343620776965646572686F6C656E21DB
:1036800020004043776572743D0014696E207469B0
:1036900065666572656E20426572656963682000C3
:1036A00014696E20686F65686572656E2042657288
:1036B000656963682000546D6974204265662E3424
:1036C00033207765636873656C6E2100542D2D2D52
:1036D0002D2057617274656E20545821202D2D2D98
:1036E0002D00542D2D2041627374696D6D756E67C8
:1036F000204F4B21202D2D00542D204E69636874DE
:103700007320676566756E64656E21202D00542DEB
:103710002D2057617274656E205458204F46462103
:10372000202D2D00542D2D2D2053617665204461D0
:1037300074656E21202D2D2D2D00544B65696E650D
:10374000204672657175656E7A2D496E666F21002F
:10375000542D2D2D204D61746368205354415254D3
:1037600021202D2D2D00542D2D2D2D204D617463E4
:103770006820454E444521202D2D2D00542D2D2D02
:103780002D204772756E646D61746368202D2D2D38
:103790002D00542D205375626D61746368202D00D7
:1037A000542D2D2D2054582041626272756368217A
:1037B000202D2D2D2D005420545820506567656C08
:1037C000207A752067726F7373212000542D204674
:1037D0006F7274736368726974743A200000250014
:1037E0000053796D54756E2E2052533233322D5260
:1037F000656D6F746500404857322E3030202020B0
:1038000032392E30342E32303232200014535731B8
:103810002E303820202028632920444C344A414C43
:103820002000544341542D50696341537461722008
:10383000444C344A414C2000544341542D465420BA
:103840003834372059616573752020202000544397
:1038500041542D4B3220456C6563726166742020A3
:1038600020202000544341542D50432D506F776544
:1038700072534452202020202000544341542D49AB
:1038800043373330302049636F6D202020202000E3
:10389000544341542D4654445831303120596165C8
:1038A0007375202020002D2D2D00494E46006D57A8
:1038B0000000755700006E570000705700006657F3
:1038C000000061570000572000006B570000205691
:1038D00000006D560000755600006E5600006442F0
:1038E0006D00644200007373000013D806D83F6A6D
:1038F000406A416A426A436A12003A6A3B6A3C6A19
:103900003D6A3E6A1200446A456A466A476A486AE6
:103910001200F9DF496A4A6A4B6A4C6A4D6A120022
:10392000596A5A6A5B6A5C6A5D6A12000EC15EF08F
:103930000FC15FF010C160F011C161F012C162F0FF
:1039400012000EC159F00FC15AF010C15BF011C145
:103950005CF012C15DF012005EC059F05FC05AF019
:1039600060C05BF061C05CF062C05DF0120059C0E5
:103970005EF05AC05FF05BC060F05CC061F05DC09B
:1039800062F0120059C00EF15AC00FF15BC010F185
:103990005CC011F15DC012F1120013C159F014C1E5
:1039A0005AF015C15BF016C15CF017C15DF0120052
:1039B00013C15EF014C15FF015C160F016C161F073
:1039C00017C162F0120018C159F019C15AF01AC19A
:1039D0005BF01BC15CF01CC15DF0120018C15EF011
:1039E00019C15FF01AC160F01BC161F01CC162F027
:1039F00012001DC159F01EC15AF01FC15BF020C159
:103A00005CF021C15DF012001DC15EF01EC15FF0CF
:103A10001FC160F020C161F021C162F0120022C11B
:103A200059F023C15AF024C15BF025C15CF026C1D6
:103A30005DF0120022C15EF023C15FF024C160F08E
:103A400025C161F026C162F0120027C159F028C1DA
:103A50005AF029C15BF02AC15CF02BC15DF0120065
:103A600027C15EF028C15FF029C160F02AC161F072
:103A70002BC162F012005EC013F15FC014F160C090
:103A800015F161C016F162C017F1120059C013F1AF
:103A90005AC014F15BC015F15CC016F15DC017F19E
:103AA000120059C018F15AC019F15BC01AF15CC07C
:103AB0001BF15DC01CF1120059C01DF15AC01EF16E
:103AC0005BC01FF15CC020F15DC021F1120059C044
:103AD00022F15AC023F15BC024F15CC025F15DC026
:103AE00026F1120059C027F15AC028F15BC029F114
:103AF0005CC02AF15DC02BF112003AC044F03BC01B
:103B000045F03CC046F03DC047F03EC048F01200D2
:103B10003AC049F03BC04AF03CC04BF03DC04CF0CD
:103B20003EC04DF0120044C03AF045C03BF046C0E4
:103B30003CF047C03DF048C03EF0120049364A36DE
:103B40004B364C364D3612004436453646364736EF
:103B5000483612004D324C324B324A324932120052
:103B600048324732463245324432120006D83F3698
:103B7000403641364236433612003A363B363C3602
:103B80003D363E36120043324232413240323F32FD
:103B90001200F9DF3E323D323C323B323A32120003
:103BA00044AE04D04568466847684868120045AE90
:103BB00003D0466847684868120046AE02D047689E
:103BC0004868120047AE01D048681200679366BF8C
:103BD00067838CDE280E376ED890B0EC1DF0CAECEF
:103BE0001DF003D8372EF8D71200B9EC27F00A0ED3
:103BF000366E00EE3AF0EF50E8B6FD0FE8BED00F9B
:103C0000EE6E362EF8D7C6EC27F012003FD83EAE47
:103C100009D03F2AD8B4402AD8B4412AD8B4422A7D
:103C2000D8B4432A7DEC1CF035D030D83EAE09D054
:103C30003F2AD8B4402AD8B4412AD8B4422AD8B4AA
:103C4000432A3FC03AF040C03BF041C03CF042C084
:103C50003DF043C03EF066BFBEEC24F0120016D823
:103C60003FC03AF040C03BF041C03CF042C03DF0A4
:103C700043C03EF066BFBEEC24F0120007D877ECDC
:103C80001CF008D003D87DEC1CF004D059EC20F0D7
:103C90004EEF1EF00BEC1FF06FEF20F04CD803E15D
:103CA00076EC1CF01AD01AD87F0E4E6E4E50525E33
:103CB0004F50535A52C036F052520FE052BE06D007
:103CC000D890B6EC1DF0362EFBD707D0361E362A1C
:103CD000D890C9EC1DF0362EFBD71200669F58BE57
:103CE000668F589E76EC1CF054C03BF055C03CF0FB
:103CF00056C03DF057C03EF058C03FF0D890B6ECEB
:103D00001DF0CAEC1DF03E8E3FC052F03F6AD890C5
:103D1000B6EC1DF01200040E366EEE6608D0362E9C
:103D2000FCD7EECFE8FF7F0B03E1D88401D0D89415
:103D3000C6EC27F01200B9EC27F000EE54F0EBD7F8
:103D4000B9EC27F000EE59F0E6D7B9EC27F000EE19
:103D50005EF0E1D7B9EC27F000EE44F0DCD7B9EC27
:103D600027F000EE49F0D7D7B9EC27F000EE3AF093
:103D70000A0E366EEE66DBD7362EFCD7D6D7486AEB
:103D800047BE486835D0476A486A46AE31D0476872
:103D900048682ED0466A476A486A45AE29D04668C8
:103DA0004768486825D0456A466A476A486A44AE0B
:103DB0001FD045684668476848681AD076EC1CF002
:103DC000669F486A1DD076EC1CF0669F476A486A79
:103DD00017D076EC1CF0669F466A476A486A10D096
:103DE00076EC1CF0669F456A466A476A486A08D0C6
:103DF00076EC1CF0669F48AE03D0CDEC24F0668FC5
:103E000044C03FF045C040F046C041F047C042F0DA
:103E100048C043F000D07F0E526E000E536EB4ECDB
:103E20001EF006E1546A556A566A576A586A36D0D7
:103E300075EC1FF007E0D890C9EC1DF0522AD8B4F9
:103E4000532AF6D73FB00AD0D890B6EC1DF05206F0
:103E50005228D8B45306D8B45252F4D73BA00BD052
:103E60003B803B2AD8B43C2AD8B43D2AD8B43E2A59
:103E7000D8B43F2ADDD73A6A3F9052C03FF0C9EC30
:103E80001DF03BC054F03CC055F03DC056F03EC064
:103E900057F03FC058F0589E66BF588E1200546AC3
:103EA000556A566A586A800E576EF5D75468556839
:103EB00056687F0E576E7F0E586EEDD77F0E446E9C
:103EC000000E456E5350455C02E15250445CD8B040
:103ED00003D0ECDFD88401D0D894120053AE03D0C5
:103EE000DEDFD88401D0D8941200B9EC27F000EEC0
:103EF00043F0040E366EED660AD0362EFCD7010E66
:103F0000EF6201D002D0EF6602D0D88401D0D894FD
:103F1000C6EC27F0120049C000F14AC001F14BC0C5
:103F200002F14CC003F14DC004F1D5EC1FF03AC0D2
:103F300007F13BC008F13CC009F13DC00AF13EC0A9
:103F40000BF100C144F001C145F002C146F003C1CC
:103F500047F004C148F0BBEC1FF007C13FF008C1B7
:103F600040F009C141F00AC142F00BC143F0669F25
:103F700067B3668F1200BADC280E376ED89005D86A
:103F8000BDEC1DF0372EFAD71200B9EC27F0050E64
:103F9000366E00EE44F0D890EF50E8200700EE6E49
:103FA000362EFAD7C6EC27F01200B9EC27F09EDCCB
:103FB000280E376ED890B0EC1DF0CAEC1DF000EE64
:103FC00044F0050E366EEFAE02D0300EEF5EEFA677
:103FD00002D0030EEF5EEE52362EF5D7372EEAD71B
:103FE000C6EC27F0120002D87DEF1DF0B9EC27F0E7
:103FF0009ADD00EE3AF010EE49F0040E366EE6500F
:10400000EE5EE650EE5A362EFCD7C6EC27F01200D4
:1040100002D87DEF1DF0B9EC27F085DD00EE3AF017
:1040200010EE49F0E650EE26040E366EE650EE2213
:10403000362EFCD7C6EC27F0120000C144F001C1B7
:1040400045F002C146F003C147F004C148F005C184
:104050004EF006C14FF0120007C149F008C14AF006
:1040600009C14BF00AC14CF00BC14DF00CC150F02E
:104070000DC151F012003BC000F13CC001F13DC048
:1040800002F13EC003F13FC004F152C005F153C03C
:1040900006F112003BC007F13CC008F13DC009F138
:1040A0003EC00AF13FC00BF152C00CF153C00DF1FC
:1040B000120059C054F05AC055F05BC056F05CC0B5
:1040C00057F05DC058F012005EC054F05FC055F06C
:1040D00060C056F061C057F062C058F0120054C082
:1040E00059F055C05AF056C05BF057C05CF058C04C
:1040F0005DF0120054C05EF055C05FF056C060F035
:1041000057C061F058C062F01200D6EC27F016E2FA
:10411000D3EC27F013E2A0EC1EF01AE0A5EC1EF0A1
:1041200017E0EBEC27F004E3A0EC1EF001E306D06F
:10413000EEEC27F006E3A5EC1EF003E313EC28F009
:104140001200EBEC27F003E308EC28F003D00DD0CD
:1041500090EC1CF05DBE03D062AF01D05D8E5DAE11
:1041600003D062BF01D05D8E12001DD8669F66BB72
:10417000667F66BD667F7AEC24F03EC000F13FC0EA
:1041800001F140C002F141C003F142C004F11ED868
:104190000BEC20F07DEC1DF08AEC1CF07F0E496EDC
:1041A000F6EC1FF01ED0669B669D5DBE668B62BFFF
:1041B000668D7FDF6EEC1EF05EDF86DF6EEC1EF03C
:1041C00069DF75EC1CF039DF2CEF20F075EC1CF08A
:1041D0004EC044F04FC045F050C049F051C04AF0C5
:1041E00012003AC052F03BC053F076EC1CF000C114
:1041F0003BF001C13CF002C13DF003C13EF004C1FF
:104200003FF00FEC1FF06FEF20F0D6EC27F009E243
:10421000D3EC27F006E2A0EC1EF006E1A5EC1EF0C0
:1042200019E113EC28F01200EEEC27F003E3EBECBD
:1042300027F0F7E2A5EC1EF010E108EC28F05DBED7
:1042400003D062AF01D05D8E5DAE03D062BF01D0FE
:104250005D8E12001DEC28F0F2D7A5DF669F66BBCD
:10426000667F66BD667F48EC25F005DFAFDFF6ECC4
:104270001FF07DEC1DF08AEC1CF07F0E496E0BECFC
:1042800020F0AFD7A5EC1EF001E11200627F00D054
:10429000D6EC27F004E2D3EC27F001E203D013ECD4
:1042A00028F01200A5EC1EF001E11200A0EC1EF0B7
:1042B00003E1ACEC1CF0120017D80BEC20F04EC060
:1042C00052F04FC053F0669F3EAE03D0668FBEECF7
:1042D00024F03AC000F13BC001F13CC002F13DC006
:1042E00003F13EC004F181D75EDFFE0E526E000E78
:1042F000536E51504F5C02E150504E5C27E013E387
:10430000502AD8B4512A5350515C02E15250505CAB
:1043100007E18AEC1CF04EC050F04FC051F016D0AF
:10432000D89018DCE6D74E2AD8B44F2A53504F5CA9
:1043300002E152504E5C07E183EC1CF050C04EF09D
:1043400051C04FF003D0D8900BDCD3D766BBCDEC77
:1043500024F066BDDCEC24F01200B7EC1CF085EF15
:1043600020F0A0EC1EF02DE05DBE2CD0D6EC27F0A6
:1043700028E2C2EC1CF0ECD848DF46EC1DF01E0E23
:10438000396E394E1ED0A1EC1CF0D8EC1CF03DDF8C
:10439000D8EC1CF07DDFDCD838DFD8EC1CF06251A3
:1043A0005D5C0BE161515C5C08E160515B5C05E1C7
:1043B0005F505A5C02E15E50595C03E046EC1DF030
:1043C000E0D7120013EC28F01200A0EC1EF008E178
:1043D0003F0E5D6E800E5C6E596A5A6A5B6A12000F
:1043E00001013F0E266F800E256F226B236B246B1D
:1043F0003F0E216F800E206F1D6B1E6B1F6B000127
:1044000051EC1DF046EC1DF022C10EF123C10FF15D
:1044100024C110F125C111F126C112F11E0E396E11
:10442000CDEC1CF004EC1DF0F0DE96EC1CF048EC3A
:1044300021F096EC1CF062515D5C0BE161515C5C1B
:1044400008E160515B5C05E15F505A5C02E15E503F
:10445000595C17E0394E15D0C2EC1CF00FEC1DF082
:104460006FD816DF67EC1DF004EC1DF04EDE5CEC3F
:104470001DF0E3EC1CF0D8EC1CF047DE46EC1DF020
:10448000CFD71200A0EC1EF008E13F0E5D6E800E4B
:104490005C6E596A5A6A5B6A120059C02CF15AC0A4
:1044A0002DF15BC02EF15CC02FF15DC030F13EEC10
:1044B0001EF03BD82ADE89DF72EC1DF02CC159F0CA
:1044C0002DC15AF02EC15BF02FC15CF030C15DF000
:1044D00046EC1EF0669566BF66853FC039F027C181
:1044E00059F028C15AF029C15BF02AC15CF02BC1F8
:1044F0005DF0395206E066A5C5D866B5D5D8392E27
:10450000FAD71200420E626F480E616F5E6A5F6AF0
:10451000606B1200400E626F490E616F0F0E606F8C
:10452000DA0E5F6EA20E5E6E1200400E626F130E08
:10453000616F5D0E606F8D0E5F6EDE0E5E6E12003F
:104540003F0E626F800E616F5E6A5F6A606B120081
:10455000400E626F5E6A5F6A606B616B1200410EB3
:10456000626F200E616F5E6A5F6A606B1200420EBE
:10457000626FC80E616F5E6A5F6A606B1200440E04
:10458000626F7A0E616F5E6A5F6A606B1200460E40
:10459000626F1C0E616F400E606F5E6A5F6A120090
:1045A000470E626FC30E616F500E606F5E6A5F6A86
:1045B0001200490E626F740E616F240E606F5E6AA6
:1045C0005F6A12004B0E626F180E616F960E606F7D
:1045D000800E5F6E5E6A12004C0E626FBE0E616FDF
:1045E000BC0E606F200E5F6E5E6A12004E0E626F30
:1045F0006E0E616F6B0E606F280E5F6E5E6A12004A
:104600003D0E626FCC0E616FCC0E606FCC0E5F6E94
:10461000CD0E5E6E12003C0E626F230E616FD70EE0
:10462000606F0A0E5F6E3D0E5E6E12003A0E626F94
:10463000830E616F120E606F6E0E5F6E980E5E6E6F
:104640001200350E626F860E616F370E606FBD0E01
:104650005F6E060E5E6E1200300E626F890E616F25
:10466000700E606F5F0E5F6E410E5E6E12002B0E5D
:10467000626F8C0E616FBC0E606FCC0E5F6E090EA8
:104680005E6E12006CDF85EF20F071DF85EF20F0A9
:1046900076DF85EF20F07BDF85EF20F081DF85EF8F
:1046A00020F087DF85EF20F05ADF05EF21F05FDF94
:1046B00005EF21F064DF05EF21F069DF05EF21F060
:1046C0006FDF05EF21F075DF05EF21F0A0EC1EF0A4
:1046D00003E113EC28F01200C2EC1CF001013F0EC4
:1046E000176F800E166F136B146B156B000128DFAC
:1046F00042EC21F051EC1DF0A1EC1CF021DF48EC64
:1047000021F05CEC1DF0E3EC1CF004EC1DF005EC7A
:1047100021F051EC1DF067EC1DF0C2EC1CF0280EEE
:10472000396ECDEC1CF014DF48EC21F046EC1DF0A6
:10473000E3EC1CF01AEC1DF085EC20F01AEC1DF0F7
:1047400085EC20F051EC1DF0D8EC1CF005EC21F0CC
:1047500096EC1CF048EC21F096EC1CF062515D5C8C
:104760000BE161515C5C08E160515B5C05E15F500D
:104770005A5C02E15E50595C05E0394E03D0C2EC50
:104780001CF0CFD7E5DE85EF20F00101276B00019B
:10479000AFEC22F048D806E354EC23F00101272BBC
:1047A0000001F6D793DFC1DE05EC21F075EC1CF0BB
:1047B00027C13FF03F5206E00BEC1FF07AEC20F0EF
:1047C00048EC21F012007ED848AE14D04DAE29D06E
:1047D0005AD848504D5C0BE147504C5C08E14650BC
:1047E0004B5C05E145504A5C02E14450495CD8B05D
:1047F00016D017D048BE02D04DBE11D044D8485074
:104800004D5C0BE147504C5C08E146504B5C05E1C8
:1048100045504A5C02E14450495CD8B002D0D8907F
:1048200001D0D88012004ED848AE14D04DAE29D059
:104830002AD848504D5C0BE147504C5C08E146508B
:104840004B5C05E145504A5C02E14450495CD8B0FC
:1048500016D017D048BE02D04DBE11D014D8485043
:104860004D5C0BE147504C5C08E146504B5C05E168
:1048700045504A5C02E14450495CD8B002D0D8802F
:1048800001D0D8901200A0EC1EF003E183EC1CF0E4
:104890000FD0D890A4EC1DF0D89047324632453264
:1048A0004432478EA5EC1EF003E18AEC1CF009D0DF
:1048B000D8909EEC1DF0D8904C324B324A3249329F
:1048C0004C8E120059C044F05AC045F05BC046F00F
:1048D0005CC047F05DC048F05EC049F05FC04AF080
:1048E00060C04BF061C04CF062C04DF0120002D8C5
:1048F0007DEF1DF0B9EC27F037D8050E366E00EECF
:1049000049F020EE3AF076EC1CF010EE44F0050E83
:10491000376E36C038F03750382638063806EF5034
:10492000E602F350DE26D9CF63F0DACF64F0F4501C
:10493000DE22E86ADE22382EFCD763C0D9FF64C0CD
:10494000DAFF372EE6D7EE5220EE3AF0060E386E3A
:104950003650385EDE52382EFDD7362ED6D7C6EC0E
:1049600027F066B30BD81200669348AE02D015D874
:1049700066734DAE02D020D8667312003A1E3B1EFD
:104980003C1E3D1E3E1E3A2AD8B43B2AD8B43C2ACF
:10499000D8B43D2AD8B43E2A1200441E451E461EF5
:1049A000471E481E442AD8B4452AD8B4462AD8B44B
:1049B000472AD8B4482A1200491E4A1E4B1E4C1ED4
:1049C0004D1E492AD8B44A2AD8B44B2AD8B44C2A06
:1049D000D8B44D2A1200C8DFB9EC27F076EC1CF0F1
:1049E000050E366E00EE49F0EE6605D0362EFCD789
:1049F000C6EC27F01200366A362AD8904DBE1CD07D
:104A000049364A364B364C364D364D50485C0BE1F4
:104A10004C50475C08E14B50465C05E14A50455C10
:104A200002E14950445CE8E276EC1CF0D8904D324B
:104A30004C324B324A3249324D50485C0BE14C50BB
:104A4000475C08E14B50465C05E14A50455C02E199
:104A50004950445C0AE34950445E4A50455A4B5021
:104A6000465A4C50475A4D50485ABDEC1DF0362E10
:104A7000DDD777DF44C049F045C04AF046C04BF06F
:104A800047C04CF048C04DF07DEC1DF0C6EF27F05C
:104A9000290E366E76EC1CF04D50485C0BE14C5004
:104AA000475C08E14B50465C05E14A50455C02E139
:104AB0004950445C0BE34950445E4A50455A4B50C0
:104AC000465A4C50475A4D50485AD880B6EC1DF0C3
:104AD000D890A4EC1DF04D50485C0BE14C50475C65
:104AE00008E14B50465C05E14A50455C02E1495003
:104AF000445C0BE34950445E4A50455A4B50465A79
:104B00004C50475A4D50485AD880362EDFD71200A5
:104B1000B9EC27F0669348AE02D03FDF668376ECAF
:104B20001CF0280E366E0A0E376E00EE3AF0EF508B
:104B30000F0B386E050E385CD8A002D0030EEF269E
:104B4000EF50F00B386E500E385CD8A002D0300E0B
:104B5000EF26EC52372EEBD7D890A4EC1DF0B6EC34
:104B60001DF0362EE0D7C6EC27F01200D6EC27F069
:104B700015E2EEEC27F01CE22FD844D85AD86795FE
:104B80001200030E636509D06467632B66B5632B5F
:104B9000030E635F6351D4EC13F01200F2DF000EDA
:104BA000F86E380EF76EA60EF66EE8EC13F01200F3
:104BB000E8DF000EF86E380EF76EAA0EF66EE8EC1F
:104BC00013F01200D6EC27F0E9E2EEEC27F0F0E269
:104BD00003D82FD867951200B9EC27F000EE43F008
:104BE00011EE31F00A0E386EEDCF36F03638376EF2
:104BF00056D836C037F053D8382EF6D7E76AC6EC09
:104C000027F01200B9EC27F0645310E001EE44F0F5
:104C100011EE44F0140E366E64C037F0E5503606DF
:104C2000372EFCD7E5CFEDFF362EFCD7C6EC27F0AC
:104C30001200B9EC27F00A0E376E64513726635123
:104C4000375CD8B002D037C063F06351645DD8A040
:104C500003D064C063F0632B6451635F6307090E84
:104C6000366E6351365E01EE31F0365204E0EECF1F
:104C7000E8FF362EFCD766A505D02B0E66BF2D0E9D
:104C80008EEC26F0668119D8669113D8645304E03F
:104C90002C0E8EEC26F009D8C6EC27F01200375007
:104CA0000F0B3009E8CFE6FF120064C038F06797B9
:104CB00006D0010E386E679702D063C038F03852C4
:104CC00026E066A106D0EFCF36F0300E365CD8A4D1
:104CD000669167A711D038C044F0020E446202D03A
:104CE00088EC26F0050E446202D088EC26F0080E0F
:104CF000446202D088EC26F0EECFE8FF66B103D024
:104D00008EEC26F002D08AEC26F0382EDAD712008C
:104D1000200E04D0200E67B5300E00D043EC13F007
:104D20001200B9EC27F00A0E366E6451365E00EEC2
:104D30003AF0EF50364E0CD0EF50364E02D0EE52D5
:104D4000F8D7EE52446E490E446409D0010E06D0E5
:104D50000F0B446E040E446402D0100EEF260A0EB0
:104D6000366E00EE3AF0EF500700EE6EE86AEF2282
:104D7000362EF9D7C6EC27F01200B9EC27F0050E55
:104D8000366E0A0E376E00EE43F0EDCF44F044501D
:104D9000F00B07E1370644500F0B03E13706362EC0
:104DA000F4D737C044F03750C6EC27F012001DECA2
:104DB00028F076EC1CF088EC25F03AC03FF03BC0C0
:104DC00040F03CC041F03DC042F03EC043F0050E13
:104DD000636F646B66956795669967971200D6EC6A
:104DE00027F044E2EEEC27F041E259EC20F04EECE3
:104DF0001EF03AC000F13BC001F13CC002F13DC0E1
:104E000003F13EC004F13FC044F040C045F041C052
:104E100046F042C047F043C048F088EC25F03AC065
:104E200007F13BC008F13CC009F13DC00AF13EC0AA
:104E30000BF100C144F001C145F002C146F003C1CD
:104E400047F004C148F0E6EC1DF007C13FF008C18F
:104E500040F009C141F00AC142F00BC143F0140E09
:104E6000636F0A0E646F669967976795669512007F
:104E7000C2EC1CF0656B5D9EA0EC1EF014E0AFEC84
:104E800022F013EC24F001E004E354EC23F0652B52
:104E9000F6D7A0EC22F0E3EC23F005E004E342ECCB
:104EA00023F06507F6D7EFEC26F0A1EC1CF05DBE11
:104EB000668F0B0E636F0A0E646F6685669912002B
:104EC000E2EC25F0650E8EEC26F0669F65BF668FDE
:104ED00065BF656D83EC1CF065C044F0D7EC26F02F
:104EE00066854BDF44C063F0E2EC25F01200CDECA8
:104EF0001CF096EC1CF042EC21F072EC1DF0F9EC89
:104F00001CF0EEEC1CF042EC21F0B7EC1CF027C1D9
:104F100059F028C15AF029C15BF02AC15CF02BC1BD
:104F20005DF005EC21F072EC1DF00FEC1DF0EEECE5
:104F30001CF042EC21F030EC1DF085EC20F096ECFA
:104F40001CF048EC21F01200B9EC27F083EC1CF0C7
:104F5000050E366E10EE3AF020EE44F0E6500F0BE0
:104F6000DF6EE638F00BDE12362EF8D7C6EC27F0EF
:104F70001200E9CF45F1EACF46F1E1CF47F1E2CFA8
:104F800048F1D9CF49F1DACF4AF1120045C1E9FF22
:104F900046C1EAFF47C1E1FF48C1E2FF49C1D9FF6D
:104FA0004AC1DAFF120064EC20F003D059EC20F083
:104FB00000D0589E7F0E58620CD0800E576207D0EA
:104FC000566605D0556603D0546601D002D0D8800D
:104FD00001D0D890120064EC20F003D059EC20F0FE
:104FE00000D0589E7F0E58620BD0800E576208D0BA
:104FF000566606D0556604D0546602D0D88001D0DB
:10500000D890120002D86FEF20F005D8588E120009
:1050100002D86FEF20F07F0E586E800E576E546AE4
:10502000556A566A120002D86FEF20F07F0E586E54
:105030005468556856685768120002D86FEF20F020
:10504000546A556A566A576A586A1200410E626F6E
:10505000A00E616F5E6A5F6A606B120026EC28F03A
:1050600005EC21F042EC22F0C2EC1CF0A0EC22F0A6
:1050700048EC21F046EC1DF0A1EC1CF0A0EC22F075
:1050800042EC21F0B7EC1CF0CDEC1CF005EC21F06B
:105090001200AAC159F0ABC15AF0ACC15BF0ADC16E
:1050A0005CF0AEC15DF054EC23F042EC22F059C04C
:1050B000B4F15AC0B5F15BC0B6F15CC0B7F15DC0E8
:1050C000B8F11200B4C159F0B5C15AF0B6C15BF0E5
:1050D000B7C15CF0B8C15DF05AEC23F082EC22F06D
:1050E00085EC20F0B1EC21F059C0BFF15AC0C0F1FD
:1050F0005BC0C1F15CC0C2F15DC0C3F11200BFC1B1
:1051000059F0C0C15AF0C1C15BF0C2C15CF0C3C16B
:105110005DF00101010EC46F000121EC23F0E3EC0E
:1051200023F009E30101040EC46F000151EC23F0E8
:1051300048EC23F018D016EC23F0E3EC23F007E35F
:105140000101030EC46F000151EC23F00CD0A0EC60
:1051500022F0E3EC23F007E30101020EC46F00012B
:1051600048EC23F000D059C0BAF15AC0BBF15BC083
:10517000BCF15CC0BDF15DC0BEF11200B4C159F01C
:10518000B5C15AF0B6C15BF0B7C15CF0B8C15DF013
:105190000101030EB96F000137EC23F0E3EC23F0BB
:1051A0000BE351EC23F051EC23F048EC23F0010128
:1051B000080EB96F00014CD02CEC23F0E3EC23F087
:1051C00009E351EC23F051EC23F00101070EB96F14
:1051D00000013ED021EC23F0E3EC23F009E351EC95
:1051E00023F048EC23F00101060EB96F000130D026
:1051F00016EC23F0E3EC23F007E351EC23F001017C
:10520000050EB96F000124D0A0EC22F0E3EC23F0EE
:1052100007E348EC23F00101040EB96F000118D038
:10522000D9EC22F013EC24F007E363EC23F0010146
:10523000010EB96F00010CD0BFEC22F013EC24F08A
:1052400007E35AEC23F00101020EB96F000100D010
:1052500059C0AFF15AC0B0F15BC0B1F15CC0B2F15E
:105260005DC0B3F11200AFC159F0B0C15AF0B1C185
:105270005BF0B2C15CF0B3C15DF0EFEC26F0050E5F
:10528000636F010E646FAFEC22F0E3EC23F003E3F5
:10529000040E646F0FD0B7EC22F0E3EC23F003E3CD
:1052A000030E646F07D0BFEC22F0E3EC23F002E3BF
:1052B000020E646F67D891EC26F0E2EC25F0B9C1DC
:1052C00044F0030E446209D0000EF86E380EF76EFB
:1052D000AE0EF66EE8EC13F054D0040E446209D022
:1052E000000EF86E380EF76EB20EF66EE8EC13F0A4
:1052F00048D0050E446209D0000EF86E380EF76EE5
:10530000B60EF66EE8EC13F03CD0060E446209D0FF
:10531000000EF86E380EF76EBA0EF66EE8EC13F06B
:1053200030D0070E446209D0000EF86E380EF76ECA
:10533000BE0EF66EE8EC13F024D0020E446209D0E3
:10534000000EF86E380EF76EC60EF66EE8EC13F02F
:1053500018D0010E446209D0000EF86E380EF76EB8
:10536000CA0EF66EE8EC13F00CD0080E446209D0B9
:10537000000EF86E380EF76EC20EF66EE8EC13F003
:1053800000D01200BDEC26F0030E446402D0010EE2
:10539000646F030E446202D0020E646F020E446218
:1053A00002D0030E646F010E446202D0040E646FDB
:1053B000000E446202D0040E646F1200BAC159F0AC
:1053C000BBC15AF0BCC15BF0BDC15CF0BEC15DF0B9
:1053D000EFEC26F0060E636F010E646FBFEC22F057
:1053E000E3EC23F002E3020E646FB7EC22F0E3EC8F
:1053F00023F002E3030E646FAFEC22F0E3EC23F042
:1054000002E3040E646FBEDF91EC26F0E2EC25F0BF
:10541000C4C144F0010E446209D0000EF86E380E8B
:10542000F76ECE0EF66EE8EC13F024D0020E446256
:1054300009D0000EF86E380EF76ED20EF66EE8EC5C
:1054400013F018D0030E446209D0000EF86E380E27
:10545000F76ED60EF66EE8EC13F00CD0040E446234
:1054600009D0000EF86E380EF76EDA0EF66EE8EC24
:1054700013F000D01200AAC159F0ABC15AF0ACC170
:105480005BF0ADC15CF0AEC15DF0EFEC26F0050E57
:10549000636F020E646F91EC26F0BDEC26F0030EF4
:1054A000446004D0040E636F020E646F020E446405
:1054B00004D0040E636F010E646F24D0AAC159F0AA
:1054C000ABC15AF0ACC15BF0ADC15CF0AEC15DF0F8
:1054D000EFEC26F0040E636F010E646F91EC26F082
:1054E000BDEC26F0030E446004D0030E636F010E82
:1054F000646F020E446406D0040E636F000E646F86
:1055000091EC26F06685E2EC25F0000EF86E380E80
:10551000F76EDE0EF66EE8EC13F01200AFC159F034
:10552000B0C15AF0B1C15BF0B2C15CF0B3C15DF083
:10553000EFEC26F0040E636F010E646FAFEC22F007
:10554000E3EC23F003E3030E646F0FD0B7EC22F01B
:10555000E3EC23F003E3020E646F07D0BFEC22F00C
:10556000E3EC23F002E3010E646F91EC26F065D8C2
:10557000E2EC25F0B9C144F0030E446209D0000EFC
:10558000F86E380EF76EAE0EF66EE8EC13F054D0EF
:10559000040E446209D0000EF86E380EF76EB20E9B
:1055A000F66EE8EC13F048D0050E446209D0000E08
:1055B000F86E380EF76EB60EF66EE8EC13F03CD0CF
:1055C000060E446209D0000EF86E380EF76EBA0E61
:1055D000F66EE8EC13F030D0070E446209D0000EEE
:1055E000F86E380EF76EBE0EF66EE8EC13F024D0AF
:1055F000020E446209D0000EF86E380EF76EC60E29
:10560000F66EE8EC13F018D0010E446209D0000EDB
:10561000F86E380EF76ECA0EF66EE8EC13F00CD08A
:10562000080E446209D0000EF86E380EF76EC20EF6
:10563000F66EE8EC13F000D01200BDEC26F0030E7D
:10564000446404D0050E636F000E646F030E446261
:1056500002D0010E646F020E446202D0020E646F2B
:10566000010E446202D0030E646F000E446202D049
:10567000030E646F1200AFC159F0B0C15AF0B1C14E
:105680005BF0B2C15CF0B3C15DF0EFEC26F0030E4D
:10569000636F010E646FAFEC22F0E3EC23F003E3E1
:1056A000020E646F11D0B7EC22F0E3EC23F003E3B9
:1056B000010E646F09D0BFEC22F0E3EC23F004E3A9
:1056C000000E646F040E636F91EC26F065D8E2EC77
:1056D00025F0B9C144F0030E446209D0000EF86E03
:1056E000380EF76EAE0EF66EE8EC13F054D0040EE2
:1056F000446209D0000EF86E380EF76EB20EF66EE8
:10570000E8EC13F048D0050E446209D0000EF86EA4
:10571000380EF76EB60EF66EE8EC13F03CD0060EBF
:10572000446209D0000EF86E380EF76EBA0EF66EAF
:10573000E8EC13F030D0070E446209D0000EF86E8A
:10574000380EF76EBE0EF66EE8EC13F024D0020EA3
:10575000446209D0000EF86E380EF76EC60EF66E73
:10576000E8EC13F018D0010E446209D0000EF86E78
:10577000380EF76ECA0EF66EE8EC13F00CD0080E79
:10578000446209D0000EF86E380EF76EC20EF66E47
:10579000E8EC13F000D01200BDEC26F0030E4464D8
:1057A00004D0040E636F000E646F030E446204D0D5
:1057B000040E636F000E646F020E446202D0010E8D
:1057C000646F010E446202D0020E646F000E4462E8
:1057D00002D0020E646F12004BC159F04CC15AF056
:1057E0004DC15BF04EC15CF04FC15DF055C15EF044
:1057F00056C15FF057C160F058C161F059C162F005
:1058000048EC21F059C04BF15AC04CF15BC04DF14E
:105810005CC04EF15DC04FF150C159F051C15AF01A
:1058200052C15BF053C15CF054C15DF05AC15EF0EF
:105830005BC15FF05CC160F05DC161F05EC162F0B0
:1058400048EC21F059C050F15AC051F15BC052F1FF
:105850005CC053F15DC054F112004BC159F04CC112
:105860005AF04DC15BF04EC15CF04FC15DF055C1C7
:105870005EF056C15FF057C160F058C161F059C188
:1058800062F042EC21F059C04BF15AC04CF15BC0C0
:105890004DF15CC04EF15DC04FF150C159F051C1A6
:1058A0005AF052C15BF053C15CF054C15DF05AC173
:1058B0005EF05BC15FF05CC160F05DC161F05EC134
:1058C00062F042EC21F059C050F15AC051F15BC076
:1058D00052F15CC053F15DC054F112004BC159F05C
:1058E0004CC15AF04DC15BF04EC15CF04FC15DF050
:1058F00055C15EF056C15FF057C160F058C161F00C
:1059000059C162F085EC20F059C00EF15AC00FF178
:105910005BC010F15CC011F15DC012F150C159F0D3
:1059200051C15AF052C15BF053C15CF054C15DF0FB
:105930005AC15EF05BC15FF05CC160F05DC161F0B7
:105940005EC162F085EC20F059C013F15AC014F129
:105950005BC015F15CC016F15DC017F14BC159F089
:105960004CC15AF04DC15BF04EC15CF04FC15DF0CF
:105970005AC15EF05BC15FF05CC160F05DC161F077
:105980005EC162F085EC20F059C018F15AC019F1DF
:105990005BC01AF15CC01BF15DC01CF150C159F035
:1059A00051C15AF052C15BF053C15CF054C15DF07B
:1059B00055C15EF056C15FF057C160F058C161F04B
:1059C00059C162F085EC20F018C15EF019C15FF09A
:1059D0001AC160F01BC161F01CC162F048EC21F0FB
:1059E00059C050F15AC051F15BC052F15CC053F143
:1059F0005DC054F10EC159F00FC15AF010C15BF0F7
:105A000011C15CF012C15DF013C15EF014C15FF012
:105A100015C160F016C161F017C162F042EC21F0CF
:105A200059C04BF15AC04CF15BC04DF15CC04EF116
:105A30005DC04FF112004BC159F04CC15AF04DC13D
:105A40005BF04EC15CF04FC15DF055C15EF056C1D8
:105A50005FF057C160F058C161F059C162F085EC48
:105A600020F059C00EF15AC00FF15BC010F15CC0BC
:105A700011F15DC012F150C159F051C15AF052C13B
:105A80005BF053C15CF054C15DF05AC15EF05BC184
:105A90005FF05CC160F05DC161F05EC162F085ECF9
:105AA00020F00EC15EF00FC15FF010C160F011C1B7
:105AB00061F012C162F048EC21F059C00EF15AC0F9
:105AC0000FF15BC010F15CC011F15DC012F155C166
:105AD00059F056C15AF057C15BF058C15CF059C13A
:105AE0005DF055C15EF056C15FF057C160F058C11E
:105AF00061F059C162F085EC20F059C013F15AC031
:105B000014F15BC015F15CC016F15DC017F15AC10C
:105B100059F05BC15AF05CC15BF05DC15CF05EC1E5
:105B20005DF05AC15EF05BC15FF05CC160F05DC1C9
:105B300061F05EC162F085EC20F013C15EF014C12B
:105B40005FF015C160F016C161F017C162F048EC5A
:105B500021F059C013F15AC014F15BC015F15CC0BB
:105B600016F15DC017F1B7EC1CF00EC159F00FC172
:105B70005AF010C15BF011C15CF012C15DF005EC90
:105B800021F059C00EF15AC00FF15BC010F15CC09A
:105B900011F15DC012F14BC159F04CC15AF04DC129
:105BA0005BF04EC15CF04FC15DF05AC15EF05BC16D
:105BB0005FF05CC160F05DC161F05EC162F085ECD8
:105BC00020F059C018F15AC019F15BC01AF15CC03D
:105BD0001BF15DC01CF150C159F051C15AF052C1C6
:105BE0005BF053C15CF054C15DF055C15EF056C12D
:105BF0005FF057C160F058C161F059C162F085ECA7
:105C000020F018C15EF019C15FF01AC160F01BC12D
:105C100061F01CC162F042EC21F013C15EF014C1CE
:105C20005FF015C160F016C161F017C162F005ECBC
:105C300021F059C050F15AC051F15BC052F15CC023
:105C400053F15DC054F10EC14BF10FC14CF110C1C5
:105C50004DF111C14EF112C14FF112004BC15FF174
:105C60004CC160F14DC161F14EC162F14FC163F1B0
:105C700050C164F151C165F152C166F153C167F180
:105C800054C168F112005FC14BF160C14CF161C1B8
:105C90004DF162C14EF163C14FF164C150F165C174
:105CA00051F166C152F167C153F168C154F112005C
:105CB00055C169F156C16AF157C16BF158C16CF118
:105CC00059C16DF15AC16EF15BC16FF15CC170F1E8
:105CD0005DC171F15EC172F1120069C155F16AC115
:105CE00056F16BC157F16CC158F16DC159F16EC1DC
:105CF0005AF16FC15BF170C15CF171C15DF172C1AC
:105D00005EF112002EEC2EF058EC2EF0ECEC2BF0A5
:105D10004BC173F14CC174F14DC175F14EC176F1B7
:105D20004FC177F150C178F151C179F152C17AF187
:105D300053C17BF154C17CF143EC2EF06DEC2EF09D
:105D40006EEC2CF073C155F174C156F175C157F169
:105D500076C158F177C159F178C15AF179C15BF137
:105D60007AC15CF17BC15DF17CC15EF11BEC2DF071
:105D70001200C8EC13F030EC2FF0D5EC11F012004B
:105D8000C8EC13F04BC159F04CC15AF04DC15BF057
:105D90004EC15CF04FC15DF05D50DAEC13F05C5029
:105DA000DAEC13F05B50DAEC13F05A50DAEC13F043
:105DB0005950DAEC13F0D2EC13F050C159F051C144
:105DC0005AF052C15BF053C15CF054C15DF05D50BC
:105DD000DAEC13F05C50DAEC13F05B50DAEC13F011
:105DE0005A50DAEC13F05950DAEC13F0400ED0ECC4
:105DF00013F055C159F056C15AF057C15BF058C164
:105E00005CF059C15DF05D50DAEC13F05C50DAECF7
:105E100013F05B50DAEC13F05A50DAEC13F05950EF
:105E2000DAEC13F0D2EC13F05AC159F05BC15AF01E
:105E30005CC15BF05DC15CF05EC15DF05D50DAECB1
:105E400013F05C50DAEC13F05B50DAEC13F05A50BC
:105E5000DAEC13F05950DAEC13F0D5EC11F0120033
:105E6000000E4BC159F04CC15AF04DC15BF04EC110
:105E70005CF04FC15DF00FD8400E50C159F051C1D8
:105E80005AF052C15BF053C15CF054C15DF003D8CD
:105E90006A0E43EF13F0D0EC13F0EFEC26F00D0E8A
:105EA000636F070E646F668591EC26F0E2EF25F0D4
:105EB000400E4BC159F04CC15AF04DC15BF04EC180
:105EC0005CF04FC15DF0E7DF140E50C159F051C1D5
:105ED0005AF052C15BF053C15CF054C15DF0DBDF9E
:105EE0006A0E43EF13F0140E4BC159F04CC15AF037
:105EF0004DC15BF04EC15CF04FC15DF0CCDF540E84
:105F000050C159F051C15AF052C15BF053C15CF01D
:0C5F100054C15DF0C0DF6A0E43EF13F0D7
:020000040030CA
:0300010022193C85
:020005003D8438
:0200000400F00A
:0400000004010100F6
:00000001FF
